:020000040800F2
:10000000D8650424BD020008334B00080F420008E5
:10001000314B00086F040008138300080000000043
:10002000000000000000000000000000FD64000867
:100030009305000800000000D54B00080167000888
:10004000D7020008D7020008D7020008D70200082C
:10005000D7020008D7020008D7020008D70200081C
:10006000D7020008D7020008D7020008D70200080C
:10007000D7020008D7020008D7020008D7020008FC
:10008000D7020008D7020008D7020008D7020008EC
:10009000D7020008D7020008D7020008D7020008DC
:1000A000D7020008D7020008D7020008D7020008CC
:1000B000D7020008D7020008D7020008D7020008BC
:1000C000D7020008D7020008D7020008D7020008AC
:1000D000D7020008D56E0008D7020008D702000832
:1000E000D7020008D702000800000000D70200086D
:1000F000D7020008D7020008D7020008D70200087C
:10010000D7020008D7020008D7020008D70200086B
:10011000D7020008D7020008D7020008D70200085B
:10012000D7020008D7020008D7020008D70200084B
:10013000D7020008D7020008D7020008D70200083B
:1001400000000000000000000000000000000000AF
:10015000D7020008D7020008D7020008D70200081B
:10016000D7020008D7020008D7020008D70200080B
:10017000D7020008D7020008D7020008D7020008FB
:10018000D7020008D7020008D7020008D7020008EB
:10019000D7020008D7020008D7020008D7020008DB
:1001A000D7020008D7020008D7020008D7020008CB
:1001B000D7020008D7020008D7020008D7020008BB
:1001C000D7020008D7020008D7020008D7020008AB
:1001D000D7020008354B0008D7020008D7020008F4
:1001E000D7020008D7020008D7020008D70200088B
:1001F000D7020008D7020008D7020008D70200087B
:10020000D7020008D7020008D7020008D70200086A
:10021000D7020008D7020008D7020008D70200085A
:10022000D7020008D7020008D7020008000000002B
:10023000D7020008D702000800000000D70200081B
:10024000D7020008D7020008D7020008D70200082A
:10025000D7020008D7020008D7020008D70200081A
:10026000D7020008D7020008D7020008D70200080A
:10027000D7020008D7020008D702000800000000DB
:10028000D702000800000000D702000800000000AC
:1002900000000000D7020008DFF80CD000F0AAF838
:1002A0000048004795880008D865042430BF72B61E
:1002B000704762B6704780F30888704706488047E9
:1002C00006480047FEE7FEE7FEE7FEE7FEE7FEE73B
:1002D000FEE7FEE7FEE7FEE7056700089902000873
:1002E0002DE9F05F0546002092469B46884606466B
:1002F000814640241BE0284641464746224600F0FE
:1003000069F853465A46C01A914110D3114618460F
:10031000224600F050F82D1A67EB01084F4622469E
:100320000120002100F047F817EB00094E41201E84
:10033000A4F10104DFDC484631462A464346BDE8C5
:10034000F09F40EA01039B0703D009E008C9121F90
:1003500008C0042AFAD203E011F8013B00F8013B7F
:10036000521EF9D27047D2B201E000F8012B491EAB
:10037000FBD270470022F6E710B513460A46044642
:100380001946FFF7F0FF204610BD30B50B46014679
:1003900000202022012409E021FA02F59D4205D324
:1003A00003FA02F5491B04FA02F52844151EA2F1CE
:1003B0000102F1DC30BD202A04DB203A00FA02F110
:1003C000002070479140C2F1200320FA03F3194343
:1003D00090407047202A04DB203A21FA02F00021E5
:1003E000704721FA02F3D040C2F120029140084345
:1003F00019467047064C074D06E0E06840F00103DF
:1004000094E8070098471034AC42F6D3FFF748FF52
:1004100014B0000834B0000870B58C1810F8015BF7
:1004200015F0070301D110F8013B2A1106D110F88D
:10043000012B03E010F8016B01F8016B5B1EF9D191
:100440002B0705D40023521E0DD401F8013BFAE717
:1004500010F8013BCB1A921C03E013F8015B01F882
:10046000015B521EF9D5A142D8D3002070BDFEE732
:10047000F0B5BFF34F8FBFF36F8F1D4900200860A9
:10048000BFF34F8FBFF36F8F1A4C216841F40031D7
:100490002160BFF34F8FBFF36F8F16497031086033
:1004A000BFF34F8F081F006843F6FF75104E1036DC
:1004B000C0F34E31C0F3C90305EA4112184642EABF
:1004C00080773760401EFAD2491EF5D2BFF34F8FB6
:1004D000206840F480302060BFF34F8FBFF36F8FF0
:1004E00003484C30016841F004010160F0BD000098
:1004F00050EF00E014ED00E02DE9F0430D4F002433
:100500001D4616468846814604EB041017F8101065
:10051000B14209D107EB40014878A84204D1891CB7
:100520004246484600F02AF8641CA4B2382CEBD3AB
:10053000BDE8F08357A500082DE9F0430E4F0024D5
:100540001D4616468846814604EB840000EB4410A5
:1005500017F81010B14209D107EB40014878A842C2
:1005600004D1891C4246484600F008F8641CA4B235
:10057000092CE9D3BDE8F0832DAD0008002310B5A8
:1005800004E011F8014B5B1C00F8014B9342F8D3D7
:1005900010BD7047F0B51C46094B0A4F164685B092
:1005A0004FF0000C10251A885B883F88121A5B1ADE
:1005B0008DE8F01092B29BB200F0A3F905B0F0BD47
:1005C000C85B0424A60100242DE9FF411C46084B0A
:1005D0001646002710251A885B88121A5B1A8DE8C8
:1005E000F00092B29BB205F0D7FFBDE8FF8100009A
:1005F000C85B04242DE9F0411546DFF85C80012238
:100600000C46064640461703394600F069FB0520B4
:1006100000F0D5F9032005F025FEC4F3074005F0EE
:1006200021FEC4F3072005F01DFEE0B205F01AFE1E
:10063000002405E0FF2005F015FE3055641CA4B22F
:10064000AC42F7D300223946404600F049FBBDE8F2
:10065000F041052000F0B3B90004025830B40C4654
:100660000178202A1AD009DC0C2A0DD0102A13D0C8
:10067000182A17D10C4801FB030108E0302A0FD0DB
:10068000402A0FD10948F6E7594301F500212046D9
:1006900030BC1A46FFF7AEBF0548ECE70548EAE76D
:1006A0000548E8E730BC70470012080000920800D7
:1006B00000080800002608000048080030B40C4676
:1006C0000146007815464A78812809D3402A07D385
:1006D000FF2A05D0FF2803D07F2A0CD2403A0BE036
:1006E0000022104603E0521C92B204F8010B9A4219
:1006F000F9D330BC7047413A8138C0B2D1B2C0EBB7
:10070000401202EB801001EB400159430C2D0CD03C
:10071000102D0CD0182D0DD0202DEAD101F560112F
:10072000204630BC1A46FFF765BF044800E0044885
:100730000144F5E701F5ED11F2E7000000140900AE
:1007400000DD1100AFF3008070B586B04FF6FF708A
:1007500003F0AAFD00206C4605462554401CC0B29B
:100760001828FAD3112220460021FFF743FF102159
:100770006B464FF4784608463246FFF70BFF0020E1
:100780002554401CC0B21828FAD308226846142108
:10079000FFF730FF20216B4610203246FFF7FAFEAC
:1007A00000202554401CC0B21828FAD308226846FD
:1007B0001E21FFF71FFF30216B4610203246FFF746
:1007C000E9FEC82008F034F806B070BD2DE9F04FFE
:1007D000C1B01C4616460D4682468946580701D0D0
:1007E000012100E0002101EBD40061080C2C10FB7A
:1007F00001F0834609D0102C07D0182C05D0202CEE
:1008000003D0302C01D0402C2DD10346224669461E
:100810003046FFF723FF002022E01DF80870002675
:10082000380601D54A9A02E04C9820B94B9A2946DD
:10083000504603F09BFD78066D1CADB2070EA5EB8C
:100840000900A04205D10AF101004D461FFA80FAC5
:1008500003E0761CB6B2082EE2D308F1010080B2A4
:1008600058458046D9D341B0BDE8F08F2DE9F04F0F
:10087000A1B01F4615460C4682468946580701D04E
:10088000012100E0002101EBD7000C2F10FB07F045
:10089000834605D0102F03D0182F01D0202F2DD143
:1008A00003463A4669462846FFF708FF002022E043
:1008B0001DF808600025300601D52A9A02E02C9820
:1008C00020B92B9A2146504603F050FD7006641C57
:1008D000A4B2060EA4EB0900B84205D10AF101004A
:1008E0004C461FFA80FA03E06D1CEDB2082DE2D3EE
:1008F00008F10100C0B258458046D9D321B0BDE807
:10090000F08F2DE9FF4F83B09B460E46044680468C
:100910008A46DDE910750020814620E0B9F1000F1C
:1009200023D005994FF0000908EB0100401BA042BD
:1009300002DA7019444686B20AEB0B00401BB04243
:1009400010DB12AB93E807002B468DE807003A4610
:1009500031462046FFF78AFF601984B2BF1C387801
:100960000028DBD107B0BDE8F08F802801D9012035
:10097000D2E7059A08EB0201A1EB5501A14202DA88
:10098000711944468EB20AEB0B01491BB142E9DBF7
:100990000D280FD012AB93E807002B468DE8070017
:1009A0003A4631462046FFF711FF04EB550084B26A
:1009B0007F1CD4E77019444686B27F1CF5E70022FD
:1009C00006E00021491CC9B26429FBD3521CD2B2F3
:1009D0008242F6D3704770B4164602781D464378BB
:1009E000812A0C4610D3402B0ED3FF2B0CD0FF2AAC
:1009F0000AD00C2D11D0102D11D0182D0DD131464B
:100A0000204670BCFFF798BD0021084603E0491C52
:100A100004F8010BC9B2B142F9D370BC704731463A
:100A2000204670BCFFF768BD10B528B190F83510AE
:100A3000022903D080214165012010BD1D4A4FF4D9
:100A4000956301688C189C4207D8042280F83520F1
:100A5000086820F00100086029E00C6824F00E040A
:100A60000C6001680A440A6822F001020A60016E03
:100A70000A6822F480720A6090F85C30012202FA5F
:100A800003F10D4B1960D0E919134B60C16E31B100
:100A90000B6823F480730B60D0E91C134B600021BA
:100AA00080F8341080F83520016D01B188470020AE
:100AB00010BD0000F0FFFDBF0454025870B504469D
:100AC00000F014F90546601C02D004480078044484
:100AD00000F00CF9401BA042FAD370BD14000024B2
:100AE0000248016841F0010101607047200400588C
:100AF0002DE9F84F6C4C00224FF0B04A4FF0010B3B
:100B00004FF0030E4FF00F090B680BFA02F73B4052
:100B1000BB4270D14D68022D01D0122D12D1D508E3
:100B200000EB850CDCF820605507ED0E09FA05F89E
:100B300026EA0806D1F8108008FA05F848EA0608FF
:100B4000CCF82080D0F80080560091F804C00EFA4E
:100B500006F50CF0030C28EA05080CFA06FC4CEA32
:100B6000080CC0F800C0D1F804C0BCF1010F08D0D7
:100B7000BCF1020F05D0BCF1110F02D0BCF1120F75
:100B800016D1D0F808C0D1F80C802CEA050C08FA70
:100B900006F848EA0C08C0F80880D0F804C02CEA2F
:100BA000070C0F79C7F30017974047EA0C07476017
:100BB000C768AF438D68B5403D43C5604D68ED00E3
:100BC0006BD53A4D2E6846F002062E602D6822F055
:100BD000030606F1B04605F002050095D6F808C4F4
:100BE00095072F0F09FA07F52CEA050C304DA8429E
:100BF00002D100252EE050E02E4DA84201D1012562
:100C000028E02D4DA84201D1022523E02B4DA8421A
:100C100001D103251EE02A4DA84201D1042519E087
:100C2000284DA84201D1052514E0274DA84201D145
:100C300006250FE0254DA84201D107250AE0244DE5
:100C4000A84201D1082505E0224DA84201D109257D
:100C500000E00A25BD4045EA0C05C6F808542568A1
:100C60004E689D43F60300D51D43256065684E68B8
:100C70009D43B60300D51D436560DAF80050564623
:100C80004F689D43FF0200D51D43356075684F686E
:100C90009D43BF0200D51D437560521C102AFFF40E
:100CA00033AFBDE8F88F000080000058F4440258CC
:100CB000000002580004025800080258000C0258B4
:100CC000001002580014025800180258001C025864
:100CD000002002580024025842694A40426170478D
:100CE0000AB1018370474183704700000148806862
:100CF0007047000014000024024881680278114403
:100D00008160704714000024032010B500F0A2F8A1
:100D1000002000F007F808B1012010BD00F06CF8C9
:100D2000002010BD70B50D4D04464FF47A7128783F
:100D3000B1FBF0F00A490968B1FBF0F003F094F858
:100D400048B9102C07D200222146501E00F062F84C
:100D500000206C6070BD012070BD000014000024F4
:100D600000000024134A41781160111D03780A1D08
:100D7000E3B143680B60017BC37A090741EA036171
:100D8000837A41EAC341437B41EA8341837B41EA61
:100D90004341C37B41EA0341437A41EA0321037A99
:100DA000007841EA43010143116070470020086068
:100DB0001060704798ED00E0BFF35F8F0448016852
:100DC00021F48031016002490020703108607047D1
:100DD00024ED00E0074940F0010008600548703844
:100DE000016841F480310160BFF34F8FBFF36F8F13
:100DF0007047000094ED00E07047002809DB0121F6
:100E000000F01F0291404009800000F1E020C0F88E
:100E1000001170470E4BF0B41B68C3F30223C3F1FB
:100E20000704042C00D904241D1D072D01D2002322
:100E300000E0DB1E012606FA04F56D1E0D409D4004
:100E40009E40761E164045EA0601F0BC07F016BC2F
:100E50000CED00E0064A00F0070110684FF6FF03B2
:100E6000184040EA01200349084310607047000021
:100E70000CED00E00000FA0501680122C0F8F8233B
:100E8000886B40F400308863886B40F4802088636E
:100E90000020704701680122C0F8F423002280F886
:100EA000EC23886940F000608861486D024A104375
:100EB000486500207047000003000010704700687C
:100EC000416200207047F0B500680023446A31B1E8
:100ED000856A4E1E04EB15444FF482750AE044EA1D
:100EE000024181620FE005EB8307C7595B1CDBB24F
:100EF00004EB1744B342F6DB4FF4807303EB81013C
:100F000044EA024242500020F0BD0000034A0121A1
:100F10001170D0F8FC0306F09FB90000EB0000242C
:100F2000C1EBC10200EB8202D0F8FC03526C06F068
:100F300009B9C1EBC10200EB8202D0F8FC03D2F880
:100F4000042206F054B90000064A002110B50446F8
:100F5000117005A007F06EFBD4F8FC03BDE810404B
:100F600006F07CB9EB0000245553422044657669B5
:100F7000636520446973636F6E6E65637465642E88
:100F80000D0A000010B504460A4601F07F000B066A
:100F9000C0EBC00104EB810101D5383101E001F55E
:100FA000FC710870D009487094F8B803012809D082
:100FB000012084F8B803206806F0C0FD002084F802
:100FC000B80310BD022010BD70B50A4604460906DC
:100FD00002F07F0005D5C0EBC00104EB8101383180
:100FE00005E0C2EBC20104EB810101F5FC710025B3
:100FF0008D700870D009487094F8B803012809D0A2
:10100000012084F8B803206806F057FF002084F818
:10101000B85370BD022070BD10B5044690F8B803F7
:1010200001280AD0012084F8B803080607D52068F3
:1010300001F07F0107F0C6F804E0022010BD20682F
:1010400007F0B0F8002084F8B80310BD01F00F01DC
:10105000C1EBC10100EB8100B0F8100280B2704713
:1010600070B504460D4601F07F000E06C0EBC001CE
:1010700004EB810101D5383101E001F5FC71ED0986
:1010800008704D708A60CB7000D0C8800025022B9C
:1010900000D10D7194F8B803012809D0012084F81B
:1010A000B803206806F0A0FC284684F8B85370BD49
:1010B000022070BD70B501F07F040D46C4EBC40181
:1010C00000EB8101C1F80C320023C1F80422C1F801
:1010D000103281F8F93181F8F84101F5FC710369AA
:1010E000012B00D10A616A06027C006803D006F079
:1010F00045FF002070BD06F021FEFAE770B50D46F1
:101100000446090605F07F0005D5C0EBC00104EBDD
:101110008101383105E0C5EBC50104EB810101F522
:10112000FC7101228A700870E809487094F8B803CD
:10113000012807D084F8B823206806F0F0FE68067E
:1011400002D007E0022070BD217C04F56F72206898
:1011500006F094FE002084F8B80370BD70B501F06D
:101160007F040D46C4EBC40100EB8101CB64002376
:101170004A640B65012381F8393001F8384F03695F
:10118000012B00D10A616A06027C006803D006F0D8
:10119000F5FE002070BD06F0D1FDFAE72DE9F84F0D
:1011A000056800260446284607F03CF800287DD153
:1011B000206807F060F8002878D0206807F05BF816
:1011C000800702D5216802204861206807F053F8A3
:1011D00001034FF0010904F56F704FF0080A009009
:1011E00077D5206807F029F8DFF8E0B480466DE095
:1011F0005FEAC87067D02068F1B207F034F807469C
:10120000C00736D005EB4611C1F8089B2A6C5A4539
:101210000AD3206901281CD1D5F8080B000406D593
:101220004FF40040C1F8080B2069012811D1C6EB2A
:10123000C600D1F8101B04EB8000D0F80022C1F3E7
:101240001201511AC0F81012D0F804121144C0F85B
:1012500004122046F1B2FFF76CFE2069012808D184
:101260003EB9D4F80C0220B920680121009A06F09A
:1012700005FE380716D5296C59450CD3206901287D
:1012800009D1D5F8080B000405D505EB46114FF43C
:101290000040C1F8080B204600F066FB05EB461144
:1012A000C1F808ABF80607D5102001E00CE210E009
:1012B00005EB4611C1F8080BB80604D505EB46113D
:1012C0002020C1F8080B761C4FEA5808B8F1000F2F
:1012D0008ED1206806F0CFFF40034FF0400B5AD567
:1012E000206806F0A3FF0026804651E05FEAC87040
:1012F0004BD02068F1B206F0A7FF0746C00724D004
:10130000D5F8341809FA06F08143C5F8341805EB0E
:101310004610C0F808992069012807D1C6EBC6001D
:1013200004EB8000D0E91021114441642046F1B261
:10133000FFF7F6FD2069012807D136B9E06C20B926
:1013400020680121009A06F099FD380703D505EBC6
:101350004611C1F808A9F80604D505EB461110207E
:10136000C1F80809780603D505EB4611C1F808B99C
:10137000B80704D505EB46110220C1F80809380664
:1013800003D53146204603F0DBFB761C4FEA5808B4
:10139000B8F1000FAAD1206806F06DFF002810DA1E
:1013A000D5F8040820F00100C5F8040894F8EC030F
:1013B000012837D0204600F0ABFA21684FF00040FA
:1013C0004861206806F057FF00050AD5D5F80808DF
:1013D000C00702D0204600F0D9FA21684FF400601F
:1013E0004861206806F047FF000109D521684FF0E9
:1013F0000060486194F8EC03E0B1204600F0C6FAC2
:10140000206806F038FFC0045FD5D5F8040820F046
:101410000100C5F804082068102106F0D3FE002062
:10142000FF221BE0002084F8EC0301462046FFF772
:1014300045FDC2E784F8EC932068406D0121C0F3BC
:101440008300C4F8F0032046FFF738FDD8E705EB2A
:101450004011C1F80829C1F8082B401C616881427D
:10146000F5D84FF0FF30C5F81808D5F81C0840F043
:101470000110C5F81C08206B60B1D5F8840840F055
:101480000B00C5F88408D5F8440840F00B00C5F8F7
:1014900044080BE0D5F8140840F00B00C5F8140818
:1014A000D5F8100840F00B00C5F81008D5F8000872
:1014B00020F4FE60C5F80008217C2068009A06F040
:1014C000DDFC21684FF480504861206806F0D3FEAF
:1014D00080047CD5206806F0C7FA2068C16821F432
:1014E0007051C160206806F07FFE78B1C4F814B076
:1014F0000320E06001F0AAFA7549764A014491425E
:101500000AD22068C16841F4705158E00020E060C0
:101510004FF40070606136E06F49704A01449142B7
:1015200004D22068C16841F4605148E06C496D4ABA
:101530000144914204D22068C16841F450513EE018
:1015400069496A4A0144914204D22068C16841F461
:10155000405134E06649674A0144914204D2206810
:10156000C16841F430512AE06349644A0144914220
:1015700004D22068C16841F4205120E06049614AEA
:101580000144914204D22068C16841F4105116E030
:101590005D495E4A0144914204D22068C16841F429
:1015A00000510CE05A4908445A4988422068C168F1
:1015B00003D241F4E05102E009E041F4C051C160BE
:1015C000204600F05FF921684FF400504861206820
:1015D00006F051FEC00636D52068816921F0100161
:1015E0008161D5F8208008F00F00C0EBC00004EB4B
:1015F0008007C8F34340022807F5FC7702D006288D
:1016000012D01BE047F6F07118EA010F16D0C8F3AC
:101610000A12F9689046284606F031FEF868404400
:10162000F860B869404408E000990822284606F0AE
:1016300026FEB969C8F30A100844B86120688169B8
:1016400041F010018161206806F015FE000705D504
:10165000204600F073F92168C1F814A0206806F054
:101660000AFEC00207D52046F1B200F055F8216805
:101670004FF480104861206806F0FDFD800207D518
:101680002046F1B200F04CF821684FF40010486198
:10169000206806F0F0FD400006D52046FFF736FC36
:1016A00021684FF080404861206806F0E4FD400763
:1016B0000AD520684568680702D52046FFF744FC34
:1016C0002068416829434160BDE8F88F0A31544FD2
:1016D000405327FF00350C00401E1BFF40420F0007
:1016E00000DC0BFF804F1200808CF9FE20D6130027
:1016F00060B6E5FE60E3160000D3CEFE40771B0027
:10170000C05BB3FEC091210000CA91FE2075380075
:10171000E05459FEE09C4100D0F8FC0305F0F0BD18
:10172000D0F8FC0305F0EEBDF0B504004FF0000763
:101730008BB054D0032084F8B903204600F060F841
:10174000206806F0F5FA04F11001684628220E46DA
:10175000FEF7F7FD94E80F0006F0A0F920680021DD
:1017600006F09DFD01250022C7EBC70004EB8000B9
:1017700080F8395080F83870C7877F1C80F83B208C
:101780000F2F02644264C264EED300204FF48273D0
:10179000C0EBC00103EB800704EB810181F8F92164
:1017A00081F8F801C88781F8FB21C1F80022C1F84F
:1017B0000422C1F80C222168CA51401C0F28E7D32B
:1017C000282231466846FEF7BCFD94E80F0006F07B
:1017D00005FA84F8B953A06A012803D005E0012076
:1017E0000BB0F0BD2046FFF755FB606A012802D11F
:1017F0002046FFF741FB206806F0E3F90020EFE701
:1018000010B5B6B004464FF48021684600914FF4FD
:101810004011219100F0D6FB17492068884229D158
:101820001648016841F00101016000682FA900F02D
:10183000010034904FF4C0502F90022030900020CF
:101840003190032032900A2033900D48FFF750F971
:101850000A480838016841F0006101600068002210
:10186000012100F0006034906520FFF7D3FA652075
:10187000FFF7C3FA36B010BD00000840E04402583C
:101880000000025870B50446C068012518B102284E
:1018900006D00AA005E010A006F0CCFE002502E06C
:1018A00014A006F0C7FED4F8FC0305F03EFDD4F802
:1018B000FC032946BDE8704005F068BD5553422041
:1018C000446576696365204C696272617279202093
:1018D0005B46533F5D0D0A005553422044657669CF
:1018E0006365204C69627261727920205B48535DA8
:1018F0000D0A000055534220446576696365204C0B
:1019000069627261727920205B46535D0D0A0000A6
:1019100010B5044604A006F08DFED4F8FC03BDE823
:10192000104005F021BD00004465766963652052D2
:101930006573756D65640D0A00000000D0F8FC0346
:1019400005F018BD10B5044690F8B803012809D079
:10195000012084F8B803206806F0B7FC002084F862
:10196000B80310BD022010BDD0F8FC2300F56F7144
:10197000104605F01BBD10B50446006806F015F9C9
:10198000206806F009FC002010BD0000064A002176
:1019900010B50446117005A006F04CFED4F8FC0307
:1019A000BDE8104005F03DBDEB00002444657669BC
:1019B000636520496E2073757370656E64206D6F6A
:1019C00064652E0D0A0000000248016841F0807134
:1019D000016070470C4802582DE9F84F17468B46B6
:1019E0000446FFF783F9824694F8400001280ED0A0
:1019F000012684F8406094F841004FF00008012867
:101A000007D0022584F840802846BDE8F88F0220E0
:101A1000FBE7C4F844804FF0020984F841900022AB
:101A2000202153462046009703F022FA0500E9D111
:101A300000225946204603F0CEF8DBF8240058B9BE
:101A40000122534602212046009703F011FA0500B7
:101A5000D8D12168C1F80C9084F84160D2E7000029
:101A6000F8B50446FFF742F907465CB194F8400028
:101A7000012809D0012684F8406094F8410000252F
:101A800020B10BE00120F8BD0220F8BD84F84050E1
:101A9000204600F051F841F28830A06420680168C7
:101AA0004FF4706393FAA3F321F47062A168B3FA60
:101AB00083F3491E99400A430260A06C0022202152
:101AC0003B460090204603F0D3F970BB4FF07F47B0
:101AD000E268E16997FAA7F763680A43216AB7FAEF
:101AE00087F7BB4019430A4321680B68104F3B40FE
:101AF0001A430A60D4E905310B4321684A684FF460
:101B0000F81C0C4F9CFAACFC3A402769BCFA8CFCE0
:101B100007FA0CF73A4313434B6021680A6842F016
:101B200001020A60656484F8416084F84050F8BDA1
:101B30002FFFFF00FEF8E0FF2D482DE9F04301687C
:101B400087B041F480410160006800F48040059056
:101B500027480C30016841F002010160016801F082
:101B600002010591016841F008010160016801F07E
:101B700008010591016841F010010160006802242C
:101B80000325DFF8709000F01000059040206946B2
:101B9000CDE900040120CDE902050A200490484661
:101BA000FEF7A6FF00264FF004080927CDF80080B5
:101BB00069464846CDE90146CDE90357FEF798FF4F
:101BC0004FF4605069468DE851000B48CDE903574A
:101BD000FEF78EFFCDF800806946CDE90146074843
:101BE000CDE90357FEF784FF07B0BDE8F08300009E
:101BF000D444025800040258000C02580010025845
:101C00002DE9F84F16460F460446FFF76FF8824657
:101C10002068816900F1200594F84020012A0ED047
:101C20004FF0010884F8408094F841204FF00009FB
:101C3000012A06D0022084F84090BDE8F88F0220E7
:101C4000FBE7C4F8449097B3222284F8412002694C
:101C5000521CA2630269521C62632763426922F02C
:101C6000406242F080624261206881610CE006219E
:101C7000204603F0FDF8B8B92A78206B411C216397
:101C80000270A06B401EA063A06B53464FF0010290
:101C900000960028EBD14FF00201204603F0E8F84F
:101CA00010B922680221D16084F84180C3E7FFE7C0
:101CB000606C40F0080060640120BCE72DE9F84F3B
:101CC00016460F460446FFF711F88246206894F83E
:101CD000401000F1200501290ED04FF0010884F8D2
:101CE000408094F841104FF00009012906D00220ED
:101CF00084F84090BDE8F88F0220FBE7C4F84490D8
:101D000077B3122184F841100169491CE16201692D
:101D1000491CA1626762416921F0406141610CE0A8
:101D20000421204603F0A4F8B8B9606A411C61623E
:101D300000782870E06A401EE062E06A53464FF087
:101D4000010200960028EBD14FF00201204603F07B
:101D50008FF810B922680221D16084F84180C7E76A
:101D6000606C40F0080060640120C1E710B500F02D
:101D7000B3FE084909684FF4807292FAA2F201F4A6
:101D80007061B2FA82F2D140034A515CC840034903
:101D9000086010BD18440258348D0008000000246B
:101DA00010B500F053FE07490968102292FAA2F21A
:101DB00001F07001B2FA82F2D140034A515CC8408E
:101DC00010BD000020440258348D0008364930B55B
:101DD0000A68096812F00302344BC1F305311B682D
:101DE000334C03F010032468DFED320AB7EE001A1B
:101DF000C4F3CC0414FB03F300EE103A2E4BB8EE00
:101E0000400A07D02D4C012A01D0022A4AD0B4FB47
:101E1000F1F10BE0244C283C22689506284A03D5B2
:101E20002468C4F3C104E240B2FBF1F101EE901A60
:101E30001968B8EE612AC1F3080101EE901A196819
:101E4000F8EE611A40EE201A31EE810A22EE000A05
:101E5000C1F34621491C00EE901AF8EE600A80EEAC
:101E6000201AFCEEC10AC0ED000A1968C1F3064150
:101E7000491C00EE901AF8EE600A80EE201AFCEE83
:101E8000C10AC0ED010A1968C1F30661491C00EEE0
:101E9000901AF8EE600A80EE201ABCEEC10A80EDBE
:101EA000020A30BD074ABFE7284402582C440258B2
:101EB0003C440258000000393844025800093D00F3
:101EC0000090D00340787D01364930B50A68096832
:101ED00012F00302344BC1F305511B68334C03F479
:101EE00080732468DFED320AB7EE001AC4F3CC0425
:101EF00014FB03F300EE103A2E4BB8EE400A07D065
:101F00002D4C012A01D0022A4AD0B4FBF1F10BE09A
:101F1000244C283C22689506284A03D52468C4F33B
:101F2000C104E240B2FBF1F101EE901A1968B8EE7B
:101F3000612AC1F3080101EE901A1968F8EE611ADE
:101F400040EE201A31EE810A22EE000AC1F346214A
:101F5000491C00EE901AF8EE600A80EE201AFCEEA2
:101F6000C10AC0ED000A1968C1F30641491C00EE20
:101F7000901AF8EE600A80EE201AFCEEC10AC0ED5D
:101F8000010A1968C1F30661491C00EE901AF8EEC7
:101F9000600A80EE201ABCEEC10A80ED020A30BD54
:101FA000074ABFE7284402582C44025844440258C8
:101FB000000000394044025800093D000090D00361
:101FC00040787D012DE9F84F0446006800252E4633
:101FD000010104F12400FE4FDFF8F88300901DD5C5
:101FE000606E50B1B0F5801F0CD0B0F5001F0ED060
:101FF000B0F5401F1DD001250FE0386840F40030D7
:10200000386016E00221201D02F056FF03E0009820
:10201000022102F0C9FF05000BD02E462088C00522
:1020200023D5606D05281ED2DFE800F00C11161BC9
:102030001B00D8F80010626E21F440111143C8F85B
:102040000010EBE7386840F40030386009E0002108
:10205000201D02F031FF03E00098002102F0A4FFF0
:1020600005466DB100E001252E432088800528D566
:10207000A06D80281ED00CDC90B140280ED114E059
:10208000D8F80010626D21F007011143C8F8001064
:10209000EBE7C02813D0B0F5807F10D001250FE00A
:1020A000386840F40030386009E00021201D02F05B
:1020B00003FF03E00098002102F076FF054685B19A
:1020C0002E432088DFF8109340052CD5D4F8A400C7
:1020D000B0F5800F20D00DDCA0B1B0F5001F0FD1FE
:1020E00015E0D8F80010A26D21F4E0711143C8F892
:1020F0000010E6E7B0F5C00F13D0B0F5000F10D018
:1021000001250FE0386840F40030386009E0002114
:10211000201D02F0D1FE03E00098002102F044FFF0
:10212000054675B12E43208800052DD5D4F8A800AA
:10213000B0F1007F21D00EDCA8B1B0F1807F10D1CA
:1021400016E0D9F80010D4F8A42021F4600111435E
:10215000C9F80010E7E7B0F1407F13D0B0F1806F0D
:1021600010D001250FE0386840F40030386009E0F5
:102170000021201D02F0A0FE03E00098002102F0E3
:1021800013FF05466DB12E43206880011FD5A06C5A
:10219000D8B110280FD0202812D0302815D0012512
:1021A00014E0D9F80010D4F8A82021F0E061114320
:1021B000C9F80010E8E7386840F40030386004E0FF
:1021C0000221201D02F078FE05466DB12E432088C5
:1021D000C0042BD5E06DB0F5005F20D00DDCA0B1C0
:1021E000B0F5805F0FD115E07A48001F0168A26C3E
:1021F00021F0300111430160E9E7B0F5405F13D0F1
:10220000B0F5804F10D001250FE0386840F4003061
:10221000386009E00021201D02F04EFE03E0009826
:10222000002102F0C1FE054685B12E4320888004BE
:1022300029D5206EB0F5403F23D010DC08B3B0F5AF
:10224000803F14D0B0F5003F0FD115E0D8F8001052
:10225000E26D21F4E0411143C8F80010E6E7B0F563
:10226000802F0ED0B0F5A02F0BD001250AE0012160
:10227000201D02F021FE03E00098012102F094FEEF
:1022800005468DB12E43208840042AD5D4F8AC00F1
:10229000B0F1405F23D010DC08B3B0F1805F14D000
:1022A000B0F1005F0FD115E0D8F80010226E21F4D4
:1022B000E0211143C8F80010E5E7B0F1804F0ED0DF
:1022C000B0F1A04F0BD001250AE00121201D02F042
:1022D000F3FD03E00098012102F066FE05466DB1B2
:1022E0002E43208800041FD5E06ED8B1B0F1805F86
:1022F0000ED0B0F1005F10D0012514E0D9F8001025
:10230000D4F8AC2021F0E0411143C9F80010E8E70F
:10231000386840F40030386004E00121201D02F0EC
:10232000CBFD05466DB12E432068C0011ED5606C03
:10233000D0B101280ED0022811D0032814D00125D5
:1023400013E0D8F80010E26E21F040511143C8F8B4
:102350000010E9E7386840F40030386004E00221FA
:10236000201D02F0A9FD054675B12E432068DFF857
:102370006CB040025AD51A48016841F4807101607E
:10238000FEF7B4FC82460EE01248001F0168626C42
:1023900021F0030111430160E8E7FEF7A7FCA0EB81
:1023A0000A0064283AD80E480068C005F5D5B5BBC8
:1023B000094818300068B4F8B01000F4407001F417
:1023C0004071884219D00448183001680AE00000C2
:1023D0002C440258504402585844025810440258A1
:1023E00000480258026821F4407142F480320260D1
:1023F000026822F4803202600160D4F8B000B0F5C7
:10240000807F22D1FEF772FC824609E0FEF76EFC67
:10241000A0EB0A0141F28830814201D9032504E092
:10242000FE4800688007F1D57DB12E432078DFF8A3
:10243000F0A3C0073CD0A06F182837D025DC78B3B4
:10244000082828D0102824D12BE0D4F8B000C0F3FD
:10245000012103290ED0DBF8001021F47C51CBF8C8
:102460000010EE480168B4F8B020C2F30B0211432B
:102470000160DBE7DBF80020EA4B22F47C5203EA40
:1024800010100243CBF80020EBE720280ED02828BC
:102490000CD001250BE00121201D02F00DFD04E010
:1024A00004E00098012102F07FFD05465DB12E4356
:1024B000207880071ED5606F062819D2DFE800F06B
:1024C000160C11161616DAF80010A26F21F038015A
:1024D0001143CAF80010EBE70121201D02F0ECFCCB
:1024E00003E00098012102F05FFD054675B100E0B0
:1024F00001252E43207840071FD5D4F890000628E8
:1025000019D2DFE800F0160C11161616DAF80010D2
:10251000626F21F007011143CAF80010EAE70121B8
:10252000201D02F0C9FC03E00098012102F03CFDEF
:1025300005469DB100E001252E43207880062BD56D
:10254000D4F88C00B0F1405F24D011DC10B3B0F1AE
:10255000805F15D0B0F1005F10D116E0D9F80010FF
:10256000D4F8902021F007011143C9F80010E4E7E6
:10257000B0F1804F0ED0B0F1A04F0BD001250AE092
:102580000021201D02F098FC03E00098022102F0D7
:102590000BFD05468DB12E43207840062BD5D4F88F
:1025A0009800B0F5406F24D011DC10B3B0F5806F07
:1025B00015D0B0F5006F10D116E0DAF80010D4F89D
:1025C0008C2021F0E0411143CAF80010E4E7B0F597
:1025D000805F0ED0B0F5A05F0BD001250AE000218E
:1025E000201D02F069FC03E00098022102F0DCFCEF
:1025F00005468DB12E43207800062BD5D4F89C00DB
:10260000B0F5C04F24D011DC10B3B0F5005F15D089
:10261000B0F5804F10D116E0D9F80010D4F898200A
:1026200021F4E0511143C9F80010E4E7B0F5004F80
:102630000ED0B0F5204F0BD001250AE00021201D5F
:1026400002F03AFC03E00098022102F0ADFC0546DE
:1026500065B32E43207800070BD5D4F88000B0F581
:10266000805F2DD0DAF8002022F440520243CAF8ED
:1026700000202078C0060BD5D4F89400B0F5807FF8
:1026800024D0D9F8002022F440720243C9F8002077
:10269000206800032CD5D4F8A000E8B1B0F5803F45
:1026A0001FD0B0F5003F21D0012520E0D9F800105F
:1026B000D4F89C2021F460411143C9F80010C9E707
:1026C0000098022102F070FC0643D2E70098022134
:1026D00002F06AFC0643DBE70021201D02F0ECFB60
:1026E00003E00098022102F05FFC054685B12E430D
:1026F0002068400322D5D4F88400B0F5801F11D0A3
:10270000B0F5001F13D0B0F5401F15D0012514E01F
:10271000D9F80010D4F8A02021F440311143C9F8B1
:102720000010E5E7386840F40030386004E00098B5
:10273000012102F039FC054655B12E432068C00343
:102740001CD5E06C70B1B0F5803F10D0012514E0CD
:10275000DAF80010D4F8842021F440111143CAF8AB
:102760000010EBE7386840F40030386004E00221E4
:10277000201D02F0A1FB0546C5B12E432068800054
:1027800004D50098022102F00FFC06432068800364
:102790001BD5E06FB8B1B0F5807F10D0B0F5007FE9
:1027A00011D0B0F5407F0ED001250DE01C4808384F
:1027B0000168E26C21F4803111430160DEE7386882
:1027C00040F40030386045B32E432068C00207D57E
:1027D000D8F80000226F20F000401043C8F8000035
:1027E0002068C00008D5DBF80010D4F8B42021F42C
:1027F00080411143CBF800102068800207D5D8F83B
:102800000010A26E21F080711143C8F800102068FA
:10281000400014D5DBF8001006E01EE070440258BA
:1028200054440258CFFFFF0021F40041CBF80010C0
:10283000DBF80010D4F8B8201143CBF80010206862
:10284000002806DA0A480168226D21F04051114340
:1028500001605EB10120BDE8F88FDAF80010E26F88
:1028600021F440711143CAF80010AEE70020F2E7EE
:102870004C4402582DE9F047DFF8BC9104460E465F
:10288000D9F8000000F00700B0420CD2D9F80010CF
:1028900021F007013143C9F80010D9F8000000F019
:1028A0000700B0427ED12078DFF89081800707D5FD
:1028B000D8F80010E26821F00F011143C8F80010A9
:1028C0002078C00762D0D8F80010A26821F47061A7
:1028D0001143C8F8001059496068183902281CD003
:1028E00003281DD0096801281DD04907002960DA96
:1028F000524F083F396821F0070101433960FEF764
:10290000F5F90546606841F28831022813D00328A2
:102910001ED001288A4627D034E009688903E5E7FC
:1029200009688901E2E7C905E0E7FEF7DFF9411B25
:10293000514501D923E08A463868C0F3C200022815
:10294000F3D123E0FEF7D2F9411B514501D916E03E
:102950008A463868C0F3C2000328F3D116E0FEF7B8
:10296000C5F9411B51450AD83868C0F3C200012897
:10297000F5D10BE0FEF7BAF9411B514502D903200E
:10298000BDE8F087386810F0380FF3D1D9F800109F
:10299000484601F00701B1420DD9016821F0070155
:1029A000314300E005E00160006800F00700B0423C
:1029B00001D00120E4E72078400707D5D8F80010BF
:1029C000226921F070011143C8F800102078010736
:1029D0001B4805D50168626921F07001114301604F
:1029E0002178C90605D50168A26921F4E061114387
:1029F00001602078800607D51149091D0868E26941
:102A000020F070001043086000F066F8D8F800105D
:102A10004FF4807292FAA2F201F47061B2FA82F27B
:102A2000D140084A515CC840074908600020FEF7C1
:102A300079F90020A4E70000002000521844025851
:102A40001C440258348D00080000002410B5FFF724
:102A50008DF908490968012292FAA2F201F00F01EA
:102A6000B2FA82F2D140044A515CC840034908607E
:102A700010BD000018440258348D000804000024E2
:102A800010B5FFF7E3FF07490968102292FAA2F296
:102A900001F07001B2FA82F2D140034A515CC840A1
:102AA00010BD00001C440258348D000810B5FFF71B
:102AB000CDFF074909684FF4807292FAA2F201F43F
:102AC000E061B2FA82F2D140024A515CC84010BDC6
:102AD0001C440258348D00083548F0B50068364D66
:102AE00010F03801334809D00411082904D0334EBE
:102AF00010290BD018290BD02046F0BD2968890673
:102B0000FBD52968C1F3C101C840F0BD3046F0BD16
:102B1000274918310A68096812F00302284BC1F3EB
:102B200005111B68274F03F001033F68DFED260AFC
:102B3000B7EE001AC7F3CC0717FB03F300EE103A09
:102B4000224BB8EE400A06D0012A01D0022A2BD02F
:102B5000B4FBF1F008E02A68920603D52A68C2F3B4
:102B6000C102D040B0FBF1F001EE900A1868B8EE57
:102B7000612AC0F3080001EE900A1868F8EE611AA5
:102B800040EE201A31EE810A22EE000AC0F3462000
:102B9000401C00EE900AF8EE600A80EE201ABCEEAF
:102BA000C10A10EE100AF0BDB6FBF1F0DCE7000040
:102BB000104402580090D0030044025840787D0130
:102BC0002C44025834440258000000393044025862
:102BD0002DE9F05F04460078DFF8FC8341F2883984
:102BE000DFF8F8A3FE4DC0074ED0D8F800104046DD
:102BF000C1F3C20102291AD00068C0F3C200032841
:102C000005D1DAF8000000F0030002280FD0606858
:102C1000B0F5803F12D010B1B0F5A02F19D02868C0
:102C200020F480302860286820F4802009E028689B
:102C3000800329D56068002874D025E0286840F416
:102C400080302860606890B1FEF750F806464F4625
:102C500009E0286840F480202860EFE7FEF746F896
:102C6000801BB8427DD828688003F7D50CE0FEF7BA
:102C70003DF806464F4604E0FEF738F8801BB842A0
:102C8000F0D828688003F7D42078D64F80075AD52B
:102C9000D8F8001040464FF47C3B11F0380F13D0A9
:102CA0000068C0F3C200032803D1DAF800008007EF
:102CB0000AD0E068A8B3296821F01901014329600E
:102CC000FEF714F806461DE02868400702D5E068C4
:102CD0000028B1D02868E16820F019000843286076
:102CE000FEF704F8064604E0FEF700F8801B022811
:102CF000B8D828684007F7D507E0FDF7F7FF801B35
:102D00000228AFD828684007F7D538689BFAABF29D
:102D100020F47C312069B2FA82F29040014339609C
:102D200011E000E0AEE0286820F001002860FDF727
:102D3000DDFF064604E0FDF7D9FF801B022891D88D
:102D400028684007F7D42078C00655D5D8F8001079
:102D500040464FF0F84BC1F3C201012917D000687B
:102D600000E0EDE0C0F3C200032805D1DAF800006E
:102D700000F0030001280AD0E069002828682CD060
:102D800040F080002860FDF7B1FF064616E0286895
:102D9000C00502D5E069802874D138689BFAABF28F
:102DA00020F0F841206AB2FA82F290400143396083
:102DB00022E0FDF79BFF801B022899D82868C005F8
:102DC000F7D538689BFAABF2216AB2FA82F220F0AA
:102DD000F8409140084338600EE020F08000286001
:102DE000FDF784FF064604E0FDF780FF801B022804
:102DF00087D82868C005F7D42078000724D5774FF6
:102E000060694C37002838680FD040F00100386006
:102E1000FDF76CFF064604E0FDF768FF801B022803
:102E20008DD838688007F7D50EE020F001003860B3
:102E3000FDF75CFF064604E0FDF758FF801B022803
:102E40007ED838688007F7D42078800623D5A0691B
:102E5000002828680FD040F480502860FDF746FF16
:102E6000064604E0FDF742FF801B022868D8286868
:102E70008004F7D50FE020F480502860FDF736FF7E
:102E8000064605E0D6E0FDF731FF801B022857D843
:102E900028688004F7D42078400744D5524F38681A
:102EA00040F480703860FDF721FF064604E0FDF72E
:102EB0001DFF801B642843D83868C005F7D5474FED
:102EC000A068483701280AD008B1052811D0386811
:102ED00020F001003860386820F0040002E0386813
:102EE00040F001003860A06888B1FDF7FFFE06469B
:102EF00009E0386840F004003860F0E7FDF7F6FEBE
:102F0000811B49451CD838688007F7D50BE0FDF7D1
:102F1000EDFE064604E0FDF7E9FE811B49450FD8AA
:102F200038688007F7D4606AF0B3D8F80010C1F3AE
:102F3000C20103297ED00228286820F0807000E0BA
:102F400079E0286003D0FDF7D1FE044687E0FDF765
:102F5000CDFE064604E0FDF7C9FE801B02287BD8A3
:102F600028688001F7D4DAF8001040F2F332914378
:102F7000E26A41EA0211A26A1143CAF8001094F809
:102F800034004FF4FE02218E4002491EA0F500706D
:102F900080B2C1F308010843218F491E02EA0141B2
:102FA000084394F83C1000E05CE0491E120202EA7B
:102FB000016108430949083108600B1D19684FF683
:102FC000F872A06C914392FAA2F2B2FA82F29040A7
:102FD00001431960014809E010440258284402588E
:102FE000004402580444025800480258001D016879
:102FF000226C21F00C01114301600168626C21F028
:10300000020111430160016841F4803101600168EF
:1030100041F400310160016841F4802101600168E0
:1030200041F001010160286840F080702860FDF7E0
:103030005DFE01E018E00FE0044604E0FDF756FEF7
:10304000001B022808D828688001F7D50AE0FDF7A0
:103050004DFE001B022802D90320BDE8F09F28681E
:103060008001F4D40020F8E70120F6E72DE9FC41C7
:1030700004460D46032084F83000A06B03285BD083
:10308000B5F5004F58D00026B5F5804F4FF40067D6
:103090004FF0806804D005B3606B40F000603FE003
:1030A000009600210196206802F0F2FD80011CD4F8
:1030B0006946204602F026FE70BB019840032DD5DC
:1030C000B4F844000104206802F09AFA20BB20689A
:1030D00002211DE0606B304322E000960021019642
:1030E000206802F0D5FD800101D53E46F2E7694631
:1030F000204602F007FE78B90198C0030ED5B4F857
:1031000044000104206802F07BFA28B920680021FD
:1031100002F0BDFA0028DDD00646DBE74646D9E7D7
:103120006063606B012658B121681348886384F896
:1031300030600120BDE8FC81606B40F08050EFE71B
:103140002B46D4E90450D4E90172042807D2A16DBA
:10315000B1F5007F03D0B1F5807F0AD00420394655
:10316000CDE90050206802F097FD84F8306000201F
:10317000E0E70220F3E70000FF0FE01FF0B5C26DAB
:10318000920F0A70C26DC2F383624A70C26DC2F3BD
:1031900001628A70C26D120CCA70B0F85C20120A0B
:1031A0000A7190F85C204A71026E120DCA80026E9C
:1031B000C2F303420A72B0F86020C2F3C0324A720E
:1031C000B0F86020C2F380328A72B0F86020C2F397
:1031D0004032CA72B0F86020C2F300320A7300268F
:1031E0004E73836B01244FF4007563B1012B3AD009
:1031F000026850499163416B41F08051416380F80E
:1032000030400120F0BDB0F86020436E9205120DF1
:1032100042EA93720A61426EC2F3C2620A75426E5A
:10322000C2F302624A75426EC2F342528A75426E1E
:10323000C2F38242CA75426EC2F3C2320A760B6989
:103240005B1C83640A7E02F00702921C9340836435
:103250000A7A02F00F0704FA07F2C264520A5343D3
:10326000C0E914350EE090F86020436E9206920A91
:1032700042EA13420A610A69521C93028364C0E95C
:1032800013534565B0F86420C2F380324A76B0F833
:103290006420C2F3C6128A7690F8642002F07F029E
:1032A000CA76826ED20F0A77826EC2F341724A7773
:1032B000826EC2F382628A77826EC2F38352CA77C9
:1032C000826EC2F3405281F8202081F82160826E24
:1032D000C2F3004281F82220B0F86820C2F3C03265
:1032E00081F82320B0F86820C2F3803281F82420CE
:1032F000B0F86820C2F3403281F82520B0F8682089
:10330000C2F3003281F82620B0F86820C2F381228F
:1033100081F82720B0F86820C2F3012281F8282024
:1033200090F86800C0F3460081F8290081F82A402F
:103330000020F0BDFF0FE01F826B0A60C26B4A6085
:10334000026C8A60426CCA60826C0A61C26C4A611B
:10335000026D8A61406DC8610020704738B5002554
:1033600004460095B0F844000104206802F09EFA7B
:1033700028B92068002102F08BFC0090284610B18B
:10338000616B014361630098C0F3432038BD0000C6
:1033900030B591B00C460546694602F0A1FE50B129
:1033A0002A6821499163696B01436963012085F8AB
:1033B000300011B030BD0098C0F38110207000982B
:1033C000C0F34010607000994FF47F40009A00EA0B
:1033D000112141EA12616180019909BA6160029983
:1033E00021720299090A61720299C1F30351A17213
:1033F000029900EA11400399C9B20843A0810398D9
:10340000C0F38520A0730398C0F30120E0730398F4
:10341000C0F303102074039800F00F006074049848
:10342000000EA0740020C4E7FF0FE01FF0B50400F9
:1034300085B036D094F83000002618B9204626769C
:1034400000F070F8032084F83000204600F048F8BF
:1034500038BB69462046FFF79BFF10BB9DF8100064
:103460009DF811104FF40075A26B6F10012A06D061
:10347000A6652046E168FFF7F9FD90B905E008432D
:1034800001D0A565F5E7A765F3E7A06DA84204D0D4
:10349000B84202D0A06B012806D1204602F0ACFC55
:1034A00010B1012005B0F0BDFDF720FC0127054655
:1034B00004E0FDF71BFC401B401C0AD02046FFF730
:1034C0004DFF0428F5D16663E66284F83070002071
:1034D000E8E74FF00040606384F830700320E1E7D4
:1034E0007CB50446FA2000210B460A46CDE90010BF
:1034F000206802F0D1FB18B9206802F0DDFB08B1AA
:1035000001207CBD204602F07FFD012520B9204628
:1035100002F010FD0028F4D084F83050616B0143B4
:103520006163EDE7194800B587B0016841F4803167
:103530000160006800F48030059014480C30016888
:1035400041F004010160016801F004010591016886
:1035500041F0080101600068694600F0080005902C
:103560004FF4F850009002200190012002900320B7
:1035700003900C2004900648FDF7BAFA042000904E
:1035800004486946FDF7B4FA07B000BDD4440258B8
:1035900000080258000C02582DE9F04F87B09946F8
:1035A00015460E460446DDF840A0FDF79FFB834616
:1035B0003EB194F83000012807D0606B40F0005015
:1035C0000DE0606B40F0006009E000206063226D58
:1035D00005EB0901914204D9606B40F00070606313
:1035E0008CE0032184F8301021680020C862A06BB1
:1035F000012800D06D0220684FF4007102F02FF80E
:10360000DFF83081012730B12268C2F83880616B61
:103610000143616370E04FF0FF3000904FEA4920B2
:1036200001909020029002200390002004900590C9
:103630006946206802F0F7F92068C16841F040014E
:10364000C160B9F1010F06D90220E0622068294665
:1036500002F09AF804E0E7622946206802F0ADF82B
:103660000028D1D11AE0406B00040ED50025206857
:1036700002F02CFB010A30707170010C000EB17069
:103680006D1CF070361D082DF1D3FDF72FFBA0EB5C
:103690000B01514523D2BAF1000F20D02068416BB5
:1036A00011F4957FDFD0C16821F04001C16020682E
:1036B000416BC90509D5B9F1010F06D9A16B0329E1
:1036C00003D002F03FF900289ED12068416B090722
:1036D00016D5C0F83880606B40F0080021E0216802
:1036E000C1F83880606B40F00040606384F830704F
:1036F000032007B0BDE8F08F84F830700120F8E7B0
:10370000416B890705D5C0F83880606B40F0020036
:1037100007E0416B890606D5C0F83880606B40F041
:1037200020006063E8E70449816384F8307000207A
:10373000DFE70000FF0FE01F3A0F00182DE9F04F00
:1037400089B09A4615460E460446DDF848B0FDF7A6
:10375000CDFA07903EB194F83000012807D0606B95
:1037600040F000500DE0606B40F0006009E0002781
:103770006763216D05EB0A00884204D9606B40F055
:103780000070606340E0032084F830002068C76266
:10379000A06B012800D06D0220684FF4007101F089
:1037A0005EFFDFF8489100284FF0010869D1401E04
:1037B00000904FEA4A20019090200497CDE902073B
:1037C00005976946206802F02EF92068C16841F02B
:1037D0004001C160BAF1010F06D92020E0622068E3
:1037E000294602F0EEF805E01020E0622068294644
:1037F00002F000F907002ED02168C1F83890606B04
:1038000038436AE084F83080012009B0BDE8F08FC9
:10381000406B400416D5002530780690717840EA58
:1038200001200690B17840EA01400690F178361DFB
:1038300040EA01600690206806A902F05DFA6D1C5E
:10384000082DE9D3FDF752FA0799411A59451FD2BD
:10385000BBF1000F1CD02068416B11F48D7FD7D0D5
:10386000C16821F04001C1602068416BC90519D5CC
:10387000BAF1010F16D9A16B032913D002F062F837
:1038800080B12268C2F83890616B01436163B9E787
:103890002168C1F83890606B3843606384F83080E9
:1038A0000320B2E72068416B090705D5C0F83890BE
:1038B000606B40F0080010E0416B890705D5C0F847
:1038C0003890606B40F0020007E0416BC90606D5F6
:1038D000C0F83890606B40F01000606392E70449D4
:1038E000816384F8308000208FE70000FF0FE01F25
:1038F0003A0F00182DE9F05F04004FF000053DD0AD
:10390000DFF8C4812068714E714F4045A36A06D02C
:10391000B04204D0B84202D0E1680F292ED8E26B41
:103920004FF0010B0BEB521CE26802F10801C908D1
:10393000404501FB0CF105D0B04203D0B84201D0A4
:1039400008291BD8404503D0B04201D0B84201D16C
:10395000102913D84FF480094B4512D1404507D0A8
:10396000B04205D0B84203D0206BB0F5702F05D817
:10397000256B05B91504B2EB154F02D90120BDE83E
:10398000F09F94F881004FF0000A20B9204684F897
:1039900080A000F09FF8022084F881002068016870
:1039A00021F001010160A069B0F1806F09D1606868
:1039B000484506D1A06B20B92068016841F48051C8
:1039C0000160A16AE0690843E16B29430843E168AB
:1039D000084321688860616A606BA2690843A16B33
:1039E000114308432169084361690843216A084378
:1039F00061680843E16C0843A1680843A16C08436F
:103A0000A16D08432168C860A06A484529D1206C8F
:103A100001282068016827D021F400410160606C12
:103A200001282068016822D021F4804101602068CB
:103A3000404506D0B04204D0B84202D0B5F5702F50
:103A400018D0404503D0B04201D0B84202D1B5F5FC
:103A5000F81F0FD0016821F4005101602168E06A6D
:103A60000864606850B119E041F40041D6E741F4C0
:103A70008041DBE7016841F40051EEE7A06A30B90C
:103A80002068816821F4C05141F4006181602068A0
:103A9000816821F4C06141F4806181602068016D1A
:103AA00021F0010101656068400206D52068C16807
:103AB000626D21F000411143C160C4F884A084F814
:103AC00081B000205BE7000000300140003800407A
:103AD000003C0040164800B5B5B0016841F0020155
:103AE0000160006800F0020034901148083001685D
:103AF00041F480410160006800F4804034904FF44C
:103B000080500090002017906846FEF75BFA4FF453
:103B100060402F900220309001203190032032909D
:103B20000520339003482FA9FCF7E2FF35B000BD14
:103B3000E0440258000402582DE9F84F044690F87A
:103B400080001F4692460A9D01288B4613D04FF0F5
:103B5000010984F88090FDF7C9F894F881200646A1
:103B60000020012A4FF480010ED062688A4209D1F8
:103B7000A2683AB902E00220BDE8F88F94F88120EB
:103B8000042A01D0022136E0BBF1000F32D0BAF195
:103B9000000F2FD077B394F88120042A02D0052299
:103BA00084F881208046C4F88400C4F864A0A4F896
:103BB0006A70A4F86870C4F85CB0A4F86270A4F8E5
:103BC000607020676067206842686FF30F023A43B5
:103BD00042602068026842F0010202606068884228
:103BE00004D12068016841F400710160E0680F2889
:103BF00040D848E0012184F880000846BCE7B4F8CA
:103C0000620070B12068416989070AD5E16D0968D1
:103C10000162E06D001DE065B4F86200401EA4F88A
:103C20006200B4F86A0080B12068416948F2080275
:103C300011420AD0006B616E0860606E001D606604
:103C4000B4F86A00401EA4F86A00681C12D0FDF7A0
:103C50004DF8801BA8420DD3204602F02BFB84F8C0
:103C60008080D4F8840040F48070C4F8840084F824
:103C70008190EBE0B4F862000028C0D1B4F86A008B
:103C80000028BCD1C8E0072849D8BDE0B4F86200DC
:103C9000F0B12068416989071AD5B4F8621001298A
:103CA0000BD9E16B49B1E16D09680162E06D001D5E
:103CB000E065B4F86200801E08E0E16D09880184C7
:103CC000E06D801CE065B4F86200401EA4F862005C
:103CD000B4F86A00E0B12068416911F4604F17D070
:103CE0004169090409D5006B616E0860606E001DB2
:103CF0006066B4F86A00801E08E0008E616E08807D
:103D0000606E801C6066B4F86A00401EA4F86A0009
:103D1000681C04D0FCF7EAFF801BA8429CD2B4F8D0
:103D200062000028B2D1B4F86A000028AED173E076
:103D3000B4F8620080B32068416989072CD5B4F8D3
:103D4000621003290CD9E16B402909D9E16D09689A
:103D50000162E06D001DE065B4F86200001F19E02B
:103D6000B4F8621001290BD9E16B49B1E16D098802
:103D70000184E06D801CE065B4F86200801E09E0FB
:103D8000E16D097880F82010E06D401CE065B4F822
:103D90006200401EA4F86200B4F86A0068B32068AC
:103DA000416911F4604F28D04169090409D5006BBD
:103DB000616E0860606E001D6066B4F86A00001FE6
:103DC00019E0416901F4C041B1F5005F09D9008EE5
:103DD000616E0880606E801C6066B4F86A00801EA8
:103DE00009E090F83000616E0870606E401C6066FB
:103DF000B4F86A00401EA4F86A00681C04D0FCF7FE
:103E000075FF801BA84289D2B4F8620000288FD1C8
:103E1000B4F86A0000288BD10022334608212046DE
:103E2000009502F0B6FA28B1D4F8840040F02000E2
:103E3000C4F88400204602F03DFA84F8808084F8BB
:103E40008190D4F8840000283FF4D8AE012093E696
:103E50004FF0E0210428086903D020F00400086135
:103E6000704740F00400FAE7401EB0F1807F10B5C3
:103E700001D3012010BD4FF0E02460610F216017D5
:103E800004F0FCFB0020A06107202061002010BD91
:103E90007047704790F8791090F87A00084370479F
:103EA00070B502680446D0691368916810F00F0F6E
:103EB00064D0594D03F490760D40354376D0C50754
:103EC00007D0DD0505D501251562E26F42F001023C
:103ED000E267820708D5CA0706D0256802222A624F
:103EE000E26F42F00402E267420708D5CA0706D033
:103EF000256804222A62E26F42F00202E2670207AA
:103F00000ED503F0200201F080552A4352EAC17217
:103F100006D0256808222A62E26F42F00802E267B2
:103F2000E26F002A3AD0800608D503F0200001F0A5
:103F30008051084302D0204602F0D0FCE06F000719
:103F400003D42068806840062AD5204602F0B8FCD9
:103F50002068816849061ED5816821F04001816092
:103F6000606FC0B12D490165606FFCF75DFD0028F1
:103F700014D0606F016DBDE870400847850615D507
:103F800003F0200501F0805635430FD02046BDE8F0
:103F9000704002F0A3BC2046FFF77BFF70BD05E038
:103FA0002046FFF776FF0020E067F7E7C6024FF0F4
:103FB00020050CD54E020AD5E803106284F879502A
:103FC00084F87A502046BDE87040FFF761BF0606CE
:103FD0000AD503F0800601F400010E4304D0204608
:103FE000BDE8704002F00ABF41060BD5590609D55D
:103FF0001168204621F04001116084F8795000F0EA
:1040000005F9CBE70002C9D55800C7D5106820F0E4
:1040100080401060C2E7000001000010AD68000899
:1040200010B5040003D094F8790010B107E0012026
:1040300010BD002084F87800204600F027F82420E6
:1040400084F879002068016821F0010101602046B0
:1040500002F080FC0128EBD0606B10B1204602F02A
:1040600093FB2068416821F4904141602068816899
:1040700021F02A0181602068016841F0010101609E
:104080002046BDE8104002F0E3BB000010B5006818
:1040900086B01B49884230D11A48016841F00101BD
:1040A0000160006800F001000590164810300168BA
:1040B00041F01001016000680121134C00F0100074
:1040C00005904FF4007000900220CDE901010390AB
:1040D0000720694604902046FCF70AFD4FF48061F2
:1040E000204600916946FCF703FD2520FCF785FE7C
:1040F000032225201146FCF78DFE06B010BD0000FE
:1041000000100140E04402580000025890F87A3054
:10411000202B4CD1B9B1B2B190F87830012B46D0F8
:10412000012380F878304166A0F86820A0F86A2062
:10413000FF228168B1F5805F07D07F2351B1B1F1D3
:10414000805F0CD010E001207047016921B940F276
:10415000FF1107E0016909BBA0F86C2004E00169C8
:10416000E1B13F21A0F86C100021C167222280F844
:104170007A2080F8781001688A6842F001028A602B
:1041800001680A6892000CD50A6842F480720A60DD
:104190000068816841F08051816006E0A0F86C30D1
:1041A000E2E7086840F49070086000207047022041
:1041B0007047000030B50068114988420CD1114A9F
:1041C0005088010408D411464FF0000344040978D4
:1041D00006D50A2901D0538030BD40F400400DE0DF
:1041E0000D2909D0084DC0F30D04401C80B2C7282A
:1041F00029555080EFD830BD40F48040508030BD0C
:10420000001001400C000024EC0300247047FEE77E
:10421000F0B500230A241F463025372610E0B4EB02
:10422000107F02D905EB107C01E006EB107C01F851
:1042300013C001EB430C00015B1C8CF80170DBB276
:104240009342ECD3F0BD0000144870B586B001680D
:1042500041F004010160016801F004010591016869
:1042600041F010010160006800260325694600F056
:104270001000059008200124CDE900060848CDE98A
:104280000245FCF735FC20206946CDE900060548CB
:10429000CDE90245FCF72CFC06B070BDE0440258A5
:1042A00000100258000802582DE9F0410D4F00247B
:1042B0000646214620467B883A8800F0BDF93D88B5
:1042C000002178884543084600F0A2F900F09CFAE6
:1042D00003E0304600F042FA641CAC42F9D3BDE87A
:1042E000F0810000C85B04242DE9F0411E4900273D
:1042F000F0222C242A252B264FF4A07338B1012854
:1043000017D002284FF0010C1BD0032822D08F7148
:104310000A804B800C8100244D818E814B880A8855
:104320000021084600F088F92046BDE8F04100F081
:104330005DB98F710B804A800C8101244D818E8183
:10434000ECE781F806C00A804B800C8102244D8185
:104350008E81E3E781F806C00B804A800C8103243C
:104360004D818E81DAE70000C85B04242DE9F0411D
:104370000B4C16460F460546608900F029FA284680
:1043800000F0ECF9A08900F023FA384600F0E6F9D5
:10439000208900F01DFA3046BDE8F04100F0DEB99A
:1043A000C85B04241A4810B586B0016841F00201C8
:1043B000016000686946174C00F00200059041F268
:1043C00003000090012001900290032003902046FA
:1043D000FCF78EFB012220461146FCF781FC0122EE
:1043E00020460221FCF77CFC012220461103FCF749
:1043F00077FC01F009FFA00401F044FF00F00CF885
:10440000012220461146FCF76BFC06B010BD0000EF
:10441000E04402580004025870B50A4D4FF480443D
:10442000002221462846FCF75BFC322004F000FA0B
:10443000012221462846FCF753FCBDE870401E20AF
:1044400004F0F6B90004025810B5FFF7ABFF00F016
:104450007BF9322004F0ECF9362000F0B9F90020A5
:1044600000F09AF93A2000F0B3F9052000F094F931
:10447000B22000F0ADF90C2000F08EF90C2000F015
:104480008BF9002000F088F9332000F085F9332003
:1044900000F082F9B72000F09BF9352000F07CF99C
:1044A000BB2000F095F9192000F076F9C02000F04B
:1044B0008FF92C2000F070F9C22000F089F901205A
:1044C00000F06AF9C32000F083F9122000F064F9CB
:1044D000C42000F07DF9202000F05EF9C62000F035
:1044E00077F90F2000F058F9D02000F071F9A420DE
:1044F00000F052F9A12000F04FF9E02000F068F937
:10450000D02000F049F9042000F046F90D2000F019
:1045100043F9112000F040F9132000F03DF92B2061
:1045200000F03AF93F2000F037F9542000F034F958
:104530004C2000F031F9182000F02EF90D2000F089
:104540002BF90B2000F028F91F2000F025F923207B
:1045500000F022F9E12000F03BF9D02000F01CF936
:10456000042000F019F90C2000F016F9112000F0D9
:1045700013F9132000F010F92C2000F00DF93F2062
:1045800000F00AF9442000F007F9512000F004F986
:104590002F2000F001F91F2000F0FEF81F2000F08E
:1045A000FBF8202000F0F8F8232000F0F5F8212097
:1045B00000F00EF9112000F00BF9782004F038F922
:1045C000292000F005F9C82004F032F90020FFF797
:1045D0008BFE012204481146FCF782FBBDE8104027
:1045E0004FF6FF70FFF760BE00040258002158B17B
:1045F000012804D0022804D0032805D103E060215B
:1046000002E0C02100E0A021362000F003B9000044
:1046100070B5084C0D460646608900F0D9F8304662
:1046200000F09CF8A08900F0D3F82846BDE870405F
:1046300000F094B8C85B04242DE9F04104460E4F05
:1046400010448846401E86B2C818401E85B278893C
:1046500000F0BEF8204600F081F8304600F07EF809
:10466000B88900F0B5F8404600F078F82846BDE873
:10467000F04100F073B80000C85B04242DE9F84F46
:104680001F460C4682468B46580700D00120790809
:1046900000EBD700203A10FB01F0002602F0FF09E2
:1046A000C0B2009040E00C2F0FD0102F11D0182F67
:1046B0003DD1204909EBC90001EB80004FF0000813
:1046C000855D280609D50A9A0BE01B4909EB4900CC
:1046D000F2E71A4901EB0910F0E70B9828B91848DE
:1046E000428821465046FFF741FE6806641C050ECD
:1046F0001448A4B24088A04219D9A4EB0B00B842D8
:1047000009D10AF101005C461FFA80FA0D480188C0
:1047100051450CD906E008F1010000F0FF08B8F19E
:10472000080FCED3761CF6B200988642BBD3BDE804
:10473000F88F0000FB970008978D00080B92000887
:10474000A4010024C85B0424012010B500F040F847
:10475000BDE81040322004F06BB8000070B50D4E7B
:104760004FF480550022044629463046FCF7B8FA3B
:10477000012230460221FCF7B3FA200A01F072FD53
:10478000E0B201F06FFD29463046BDE870400122DD
:10479000FCF7A6BA0004025870B50C4D4FF48054D3
:1047A0000022064621462846FCF79AFA01222846AE
:1047B0000221FCF795FA304601F054FD21462846C7
:1047C000BDE870400122FCF78BBA000000040258DB
:1047D00070B50C4E4FF480550022044629463046F1
:1047E000FCF77EFA002230460221FCF779FAE0B2AB
:1047F00001F038FD29463046BDE870400122FCF743
:104800006FBA00000004025801480089FFF7E0BFBA
:10481000C85B042410B50C46FFF7DAFFE0B2BDE830
:104820001040FFF7B9BF00000E4810B586B0016810
:1048300041F001010160006869460B4C00F0010085
:104840000590022000900120019002900320039027
:104850002046FCF74DF9012220460221FCF740FAE0
:1048600006B010BDE0440258000002580EB5002109
:10487000012000900323CDE90101122102464806E0
:1048800000F001F80EBD2DE9FF4707461E460CA8B3
:1048900014460D4690E80007FCF78EFA01208DF8CB
:1048A000000000208DF808508DF80C008DF80900EC
:1048B0008DF80D808DF80A0068468DF80E908DF801
:1048C000014001978DF80B608DF80FA0FCF74AFAB4
:1048D0000420FCF77FFA04B00020BDE8F08770B533
:1048E000D0F81842054604F50041087E38B94869F9
:1048F00028B1607A18B90121284602F084FD81218F
:10490000284602F080FD607A022809D148F20C00A6
:1049100022182846BDE870401F23012102F0FEBC8A
:1049200070BD000070B5D0F818420646012104F5AC
:1049300000452869286368696863304602F0A0FC76
:104940001F280AD12649E868884206D1697E0129D4
:1049500003D8A87E08B1102808D9697E2023052233
:10496000304600F0CEFD022060720AE048F21B00E3
:104970002218304600F0A2FB0028207A08DA052829
:1049800004D03046BDE87040FFF7A9BF012121E007
:10499000022824D0012822D0032820D06389C3B163
:1049A000D6F8185204F10C02304605F500414C6966
:1049B0009C4200D223464C6B9BB2E41A4C63002409
:1049C00081F8384004212972BDE87040812102F04D
:1049D00031BD00213046BDE8704000F089B870BD9F
:1049E0005553424310B5D0F81842627A022A08D0D3
:1049F00009060BD5012A09D0BDE81040012100F0BD
:104A000077B8812102F0FFFC0020607210BD10B564
:104A1000D0F818220446117A022905D0032901D0C2
:104A2000042911D100210BE048F21900815C801C9F
:104A30000244204600F042FB002805DA012120460E
:104A4000BDE8104000F054B810BD10B5D0F81822E1
:104A50000446117A89B1012913D148F21900815C09
:104A6000801C0244204600F029FB002809DA204679
:104A7000BDE81040012100F03BB8BDE81040FFF751
:104A800051BF10BDD0F8180200210172704770B5F7
:104A9000D0F818420546002104F5004021726172E9
:104AA00080F85D1080F85C10D5F81C0201680020C9
:104AB00088470121284602F0DCFB8121284602F0CC
:104AC000D8FB48F20C0022182846BDE870401F238E
:104AD000012102F023BCD0F8181200221F230A7211
:104AE00001224A7248F20C020A44012102F016BC6B
:104AF00070B5D0F8184205460C480D2304F5004265
:104B0000D062002082F838108121207248F22C00F7
:104B10002218284602F08EFC48F20C002218284683
:104B2000BDE870401F23012102F0F8BB55534253EA
:104B3000FEE770470148FCF731BB000040560424F3
:104B40002DE9F84F0E46D0F800808146C1EBC60132
:104B500000EB8104D4E91301451A206C3834A842D3
:104B600000D20546E81C08EB461AC11700EB91700D
:104B7000871018E0451AA068A84200D20546E81C34
:104B8000ABB2C117F2B200EB9170871099F8100028
:104B900000904046E16803F0A9FBE0682844E0602B
:104BA000A0692844A061DAF8180980B2B84205D992
:104BB000D4E90501814201D20028DBD1002D06DCB9
:104BC0000120D8F83418B0408143C8F834180020C8
:104BD000BDE8F88F7047F0B54B6A4FF040652BB1D8
:104BE000AA4203D004688B6A5B1E23614FF4F8036A
:104BF0008C69002C72D00E6ACEB306688C68F461A2
:104C0000CC69F4B1D1E90B67D1F824C093FAA3F3CE
:104C10003E434F6BB3FA83F347EA0C073E434F69B9
:104C20009F400B693E431E430B6A1E43CB681E43E5
:104C30008B6926431E430B686FE0006849688161F9
:104C4000F0BDD1E90B454E6A93FAA3F32C434D6BAB
:104C5000B3FA83F335432C434D699D400B692C43D4
:104C60001C430B6A1C438B6909681C436AE0FFE71D
:104C7000CE690EB3D1E90B7CD1F824E093FAA3F30B
:104C800047EA0C07D1F834C0B3FA83F34CEA0E0CB0
:104C900047EA0C07D1F814C00CFA03FCCB6847EACA
:104CA0000C071F430B68374327431F430368174311
:104CB0005F61AA42C1D1F0BDD1E90B564F6A93FAA8
:104CC000A3F335434E6BB3FA83F33E4335434E694A
:104CD00009689E403543254362E0FFE70C6AB4B3A0
:104CE00006688C68F461CC69CCB1D1E90B67D1F866
:104CF00024C093FAA3F33E434F6BB3FA83F347EA1E
:104D00000C073E434F699F400B693E431E430B6AAD
:104D10001E43CB681E438B6926431E432DE0D1E919
:104D20000B454E6A93FAA3F32C434D6BB3FA83F30E
:104D300035432C434D699D400B692C431C430B6A42
:104D400089691C4300680C4314434461F0BDFFE7CC
:104D5000CC69B4B1D1E90B67D1F824C093FAA3F3BD
:104D60003E434F6BB3FA83F347EA0C073E434F6968
:104D70009F40CB683E431E432643036816435E6153
:104D800097E74C6A002CE1D0D1E90B5693FAA3F3D4
:104D900035434E6B4969B3FA83F326433543994053
:104DA00000680D4315434561D0E700000F480E49E8
:104DB00010B5016001214160042181601021C160B2
:104DC000C90491FAA1F1B1FA81F1491E01614FF4D0
:104DD0008061416100218161C1610162FCF740FE97
:104DE000002800D0012010BD00500052D41500242E
:104DF000074A491E10B51268116141F28832014616
:104E00000348FCF7FDFE002800D0012010BD000083
:104E1000D415002470B58EB00DF1480C9CE87000DC
:104E2000CDE9000100200395099669460D90CDE972
:104E300007400B900C90CDE90523034841F28832DE
:104E4000FCF7CAFD0EB070BDD4150024074A491EF8
:104E500010B51268116141F2883201460348FCF72F
:104E60002DFF002800D0012010BD0000D415002423
:104E70002DE9F0411E46174688460546069C11E07E
:104E8000601C0FD024B1FBF731FF801BA04209D971
:104E9000042085F84100686C40F00100686401203E
:104EA000BDE8F0812868806810EA080000D0012081
:104EB000B842E5D10020F3E72DE9F047DFF8E480C0
:104EC00004460F464FF00009D8F80000C0438007A1
:104ED00009D0344D283D286820F080602860FBF719
:104EE00005FF064607E00120BDE8F087FBF7FEFE60
:104EF000801B02284ED828680001F7D4D8F800108B
:104F0000226821F47C3141EA0231C8F80010207A8D
:104F10004FF4FE02A1884002491EA0F5007080B245
:104F2000C1F308010843A189491E02EA014108436F
:104F3000217C1202491E02EA01610843194910311D
:104F400008601848001D0168626921F0C001114322
:104F500001600168A26921F02001114301606FB175
:104F60000168012F0ED041F400110160286840F063
:104F700080602860FBF7BAFE04460DE0016841F44A
:104F80000021F2E741F48011EFE7FBF7AFFE001BD1
:104F9000022801D90320A7E728680001F5D5484673
:104FA000A2E70000284402582DE9F047DFF8E4802A
:104FB00004460F464FF00009D8F80000C0438007B0
:104FC00009D0344D283D286820F080502860FBF738
:104FD0008DFE064607E00120BDE8F087FBF786FE60
:104FE000801B02284ED828688000F7D4D8F800101B
:104FF000228821F07C7141EA0251C8F80010207A21
:105000004FF4FE02A1884002491EA0F5007080B254
:10501000C1F308010843A189491E02EA014108437E
:10502000217C1202491E02EA016108431949183124
:1050300008601848001D0168626921F4406111434D
:1050400001600168A26921F40071114301606FB130
:105050000168012F0ED041F080710160286840F096
:1050600080502860FBF742FE04460DE0016841F4E1
:105070008001F2E741F40001EFE7FBF737FE001B88
:10508000022801D90320A7E728688000F5D5484603
:10509000A2E700002844025810B5D0F818421A447C
:1050A00004F50044236E9A4206D92123052200F01C
:1050B00028FA4FF0FF3010BD002010BD2DE9F0415F
:1050C000137800244FF0FF35232B6ED00DDC1A2B04
:1050D0006CD005DCBBB1032B37D0122B11D166E0AD
:1050E0001B2B01D01E2B0CD184E02A2B76D004DCA4
:1050F000252B74D0282B04D1A6E02F2B70D05A2B4F
:105100006FD02023AEE0D0F818720646884607F527
:105110000040416931B1417E20230522304600F034
:10512000F0F9ABE0D6F81C0281684046884740B1F0
:105130003A2341460222304600F0E3F90520387256
:105140009CE020467C81BDE8F081D0F81812002355
:105150002046CC185B1CDBB2122B2073F9D37023D2
:105160000B730C23CB7401F5004393F85C4093F868
:105170005D50AC4212D001EBC4053C3505F500454D
:10518000641CE4B22E78042C8E736E790E762D7921
:105190004D7683F85C4001D183F85C0012234B818B
:1051A0001279122ACFD84A81CDE745E027E0557819
:1051B000D0F81832ED0702D0334907200CE0D0F8C0
:1051C0001C0201EBC1011279C06900EB8101087971
:1051D000401D824200D81046588108E038E02FE098
:1051E0003AE01AE0401E80B21D180A5C2A730028BB
:1051F000F8D11FE0D0F8181220464C81A3E7D0F870
:1052000018120820214A4881401E0004000C01EBBE
:105210000005135C2B73F7D10CE0D0F818020821BD
:105220001B4A4181491E0904090C00EB0105535C2E
:105230002B73F7D1204686E7BDE8F04100F02AB98C
:10524000BDE8F04100F0F8B8BDE8F04100F0A7B8C3
:10525000BDE8F04100F076B95278D0F818629207B4
:1052600002D5242305225AE706F50042B2F8683039
:10527000526E9BB2FFF710FF002801DA284662E762
:10528000204674815FE70000808D0008878D00084C
:105290008F8D00082DE9F047D0F8186207464FF4CB
:1052A0000040884606F50044A56E854200D30546B9
:1052B000B4F85E00B5FBF0F18BB2616EB1FBF0F2B9
:1052C000D7F81C0206F10C018946D0F810C0404600
:1052D000E047002809DA112341460422384600F04D
:1052E00010F94FF0FF30BDE8F087ABB24A4681219C
:1052F000384602F09FF8606E28446066A06E401B3E
:10530000A066616BA1EB0501616301D103203072DE
:105310000020E8E72DE9F0478846D0F818124FF44E
:105320000046074601F50044A56EB54200D3354658
:10533000B4F85E000C31B5FBF0F2894693B2626EB0
:10534000B2FBF0F2D7F81C02D0F814C04046E04798
:10535000002809DA032341460422384600F0D1F838
:105360004FF0FF30BDE8F087606E28446066A06EA5
:10537000401BA066616BA1EB050161630AD0B042DE
:1053800000D330464A4683B23846012101F0C6FFB9
:105390000020E7E700213846FFF7AAFBF8E72DE9F0
:1053A000F047D0F81852074616468946287AC8BBF7
:1053B00005F500444FF0FF38207E00062ED5D7F8C3
:1053C0001C0281684846884730B13A234946022288
:1053D000384600F096F811E0D6F80200494600BAC7
:1053E00020F0FF02707902436266B6F8070043BA04
:1053F0003846A366FFF750FE002802DA4046BDE8B3
:10540000F08702202872B4F85E10606E4843606630
:10541000A06E4843A0666169814204D02023617E6A
:105420000522D5E7FFE74FF400404946688138463A
:10543000BDE8F047FFF72EBF70B505460E46D5E92B
:105440008640436848F25E002218801C21183046CE
:10545000984740B13A2331460222284600F051F8DD
:105460004FF0FF3070BD04F50041086E401E020E83
:105470002273020C6273020AA273E073002020748C
:105480006074B1F85E00010AA174E07408206081C4
:10549000002070BD2DE9FC41D0F8184206460020DE
:1054A0000F4605462118401C80B20C280D73F9D315
:1054B000D6F81C0201A96A4643683846984748B1A5
:1054C0003A2339460222304600F01BF84FF0FF30F5
:1054D000BDE8FC810820E0730198401E010E217494
:1054E000010C6174010AA174E074022020756575D5
:1054F000BDF80000010AA175E0750C206081002054
:10550000E6E710B5D0F8181201F5004090F85D40BC
:1055100001EBC40404F5004484F83C201A0290F81E
:105520005D3001EBC30101F500410A6490F85D10A4
:10553000491CC9B280F85D10042902D1002180F80D
:105540005D1010BD2DE9F047D0F8185206461746F9
:105550008946287A20B13046BDE8F047FFF7DABE29
:1055600005F500444FF0FF38207E000635D4D6F80C
:105570001C0281684846884728B13A230AE0304631
:10558000FFF7BFFF1BE0D6F81C02C16848468847FA
:1055900018B1272349460222F1E7D7F8020049460D
:1055A00000BA20F0FF02787902436266B7F807007C
:1055B00043BA3046A366FFF76FFD002802DA404683
:1055C000BDE8F087B4F85E10606E48436066A06E78
:1055D0004843A0666169814203D02023617E052291
:1055E000CDE701212972C903884200D3084683B25E
:1055F0003046012105F10C0201F090FE0020DFE7AA
:1056000010B586B0044600200091372101914FF477
:105610008071CDE90210080169460490204600F02F
:1056200059FB372141F28832204600F00FFA06B0CC
:1056300010BD10B586B004460020009129210191CB
:105640004FF48071CDE902100801694604902046AC
:1056500000F040FB204600F0B1FA06B010BD10B5D6
:1056600086B0044600200091102101910901CDE986
:105670000210080169460490204600F02BFB10211F
:1056800041F28832204600F0E1F906B010BD10B5B5
:1056900086B0044600200091062101914FF48071EC
:1056A000CDE90210080169460490204600F012FB83
:1056B000062141F28832204600F0C8F906B010BD3C
:1056C00030B585B00446002569464FF480500095FA
:1056D00001950295CDE90350204600F0FBFA0B48F6
:1056E0004FF4FA510068B0FBF1F141F288304143C8
:1056F000491E02D24FF0004504E0606B0006F7D56A
:105700000348A06305B0284630BD00000000002417
:10571000C500200030B585B004464FF4D570694609
:1057200000250090082001904001CDE9020500010C
:105730000490204600F0CEFA12484FF4FA51006867
:10574000B0FBF1F041F288314843401E03D24FF0E4
:10575000004005B030BD616B11F0450FF5D0606BB6
:10576000400701D5042003E0606BC00702D0012090
:10577000A063EEE7606B400601D54020A063284699
:10578000E7E700000000002410B586B004460020C2
:105790000091122101914FF48071CDE902100801AE
:1057A00069460490204600F095FA122141F28832B1
:1057B000204600F04BF906B010BD10B586B0044687
:1057C00000200091112101914FF48071CDE9021068
:1057D000080169460490204600F07CFA112141F24C
:1057E0008832204600F032F906B010BD10B586B000
:1057F00004464FF4807007210092CDE9011000208B
:1058000003904FF4805069460490204600F062FAFD
:10581000072141F28832204600F018F906B010BD89
:1058200010B586B00446002102224FF44070CDE945
:105830000201D0020490CDE900126946204600F032
:1058400049FA204600F092F906B010BD10B586B0B6
:10585000044600200091092101914FF44071CDE9E7
:1058600002104FF4805069460490204600F032FA4E
:10587000204600F07BF906B010BD10B586B0044696
:10588000002133224FF48070CDE902010001049021
:10589000CDE900126946204600F01CFA332141F29E
:1058A0008832204600F0D2F806B010BD10B586B0A0
:1058B0000446002000910D2101914FF48071CDE943
:1058C0000210080169460490204600F003FA0D21F9
:1058D00041F28832204600F0B9F806B010BD30B56C
:1058E00085B0054603200C4600236946CDE900300B
:1058F0004FF48070CDE9020300010490284600F0C7
:10590000E9F903212246284600F07AF905B030BDB6
:1059100010B586B0044600210D224FF48070CDE909
:10592000020100010490CDE900126946204600F012
:10593000D1F90D2141F28832204600F087F806B0F7
:1059400010BD000010B50C21044686B00020CDE942
:1059500000014FF48071CDE9021008010490E06865
:1059600040F08000E060E06820F04000E0606946C0
:10597000204600F0AFF9054A0C21204600F066F8F9
:10598000E16821F08001E16006B010BD00E1F5059D
:1059900010B586B0044600200091062101914FF415
:1059A0008071CDE90210080169460490204600F09C
:1059B00091F9062141F28832204600F047F806B0FE
:1059C00010BD10B586B00446002000911921019148
:1059D0004FF48071CDE90210080169460490204619
:1059E00000F078F9192141F28832204600F02EF8B3
:1059F00006B010BD10B586B00446002000911821F5
:105A000001914FF48071CDE90210080169460490BC
:105A1000204600F05FF9182141F28832204600F05C
:105A200015F806B010BD0A6842624A688262D1E980
:105A300002231A43D1E904310B43C16A1A4321F00E
:105A4000FF011143C162002070470000444B10B5B4
:105A50004FF4FA541B68B3FBF4F35343414A5B1E03
:105A600002D24FF0004010BD446B1442F7D0426B9D
:105A7000520703D504218163084610BD426BD2074B
:105A800002D00121816306E0364A803282630269D6
:105A9000D2B28A4201D0012010BD002100F0F8F8F6
:105AA0003149084201D1002010BD002802DA4FF030
:105AB000007010BD410001D5402010BD810001D50E
:105AC000802010BDC10002D54FF4807010BD0101CF
:105AD00002D54FF4007010BD410102D54FF4806033
:105AE00010BDC10102D54FF4006010BD010202D506
:105AF0004FF4805010BD410202D54FF4005010BD4C
:105B0000810202D54FF4804010BDC10202D54FF48E
:105B1000004010BD410302D54FF4003010BD810399
:105B200002D54FF4802010BDC10302D54FF40020F0
:105B300010BD010402D54FF4801010BD410402D500
:105B40004FF4001010BD810402D54FF4800010BD49
:105B5000000702D54FF4000010BD4FF4803010BD97
:105B6000000000244500200008E0FFFD11494FF42B
:105B7000FA520968B1FBF2F141F288325143491EF1
:105B800002D24FF000407047426B12F0450FF6D042
:105B9000416B490703D50421816308467047416B77
:105BA000C90703D001218163084670470249816318
:105BB0000020704700000024C50020000E494FF46B
:105BC000FA520968B1FBF2F141F288325143491EA1
:105BD00002D24FF000407047426B12F0450FF6D0F2
:105BE000416B490703D50421816308467047034987
:105BF000816300207047000000000024C5002000E1
:105C00001F4B10B54FF4FA541B68B3FBF4F341F289
:105C1000883463435B1E02D24FF0004010BD446BDA
:105C200014F0450FF6D0436B5B0703D50421816365
:105C3000084610BD436BDB0702D00121816303E0FE
:105C40000369DBB28B4201D0012010BD0D49816395
:105C5000002100F01DF810F4604F04D0410406D577
:105C60004FF4005010BD000C1080002010BD000447
:105C700002D54FF4805010BD4FF4803010BD0000AD
:105C800000000024C5002000006800F003007047F9
:105C9000084440697047000030B51143DDE9034511
:105CA0004268234319432943024B1A400A43426086
:105CB000002030BD002CFCFF10B5016841F003014D
:105CC00001600220FAF7FAFE002010BDD0F8800033
:105CD000704700000A688260D1E901231A43D1E9C4
:105CE00003310B43C1681A43024B19401143C16091
:105CF00000207047C0E0FEFF0968C0F88010002057
:105D0000704700002DE9F04F87B00E460446FAF7C1
:105D1000EDFF002581462F4620680821B846FFF791
:105D20009EFC00283CD1B4F8440001042068FFF731
:105D300067FC002834D14FF0080A4FF0020B401ED8
:105D40006946CDE9000A3020CDE9020B0120CDE9FA
:105D500004702068FFF767FE2068FFF78EFD0028BB
:105D60001ED111E0416B090308D43DB9FFF7AEFF26
:105D700007462068FFF7AAFF01258046FAF7B6FF1D
:105D8000A0EB0900401C0ED02068416B40F22A5263
:105D90001142E7D0416B090708D5C0F838A00820A8
:105DA00007B0BDE8F08F4FF00040F9E7416B89077D
:105DB00003D5C0F838B00220F2E7416B890603D55D
:105DC000202181630846EBE70449816398FA88F053
:105DD000306038BA70600020E2E700003A0F001827
:105DE000044810B5FDF7BAFA042801D0012010BD0F
:105DF000002010BD340500242DE9F04F97B0054672
:105E000040214FF000086846FAF7B4FA0026FAF786
:105E10006DFF8146A86D18B1B0F5807F05D065E0B3
:105E20004FF0806017B0BDE8F08F28680024C4628E
:105E300040212868FFF713FC0028F3D1401E4FF0E3
:105E4000020A4FF0010B1090402011906020CDE924
:105E5000120ACDE9144B286810A9FFF7E4FD10B130
:105E60004FF48030DEE722492868FFF791FD5FEAB2
:105E70000008D7D16F462968486B40F22A52104279
:105E80001AD1486B00040BD500242868FFF71EFFC9
:105E900004EBC601641C082C47F82100F5D3761CDE
:105EA000FAF724FFA0EB0900401CE4D14FF00040BA
:105EB000686385F830B0B5E7486B000703D5082064
:105EC00088630020AEE7486B800701D5504603E0A9
:105ED000486B800602D520208863A3E705488863C5
:105EE0009DF80D00800701D44FF08058404699E797
:105EF00001FFFF80FF0FE01F0D484FF480420B4968
:105F000010B5016000214160C0E902120161042165
:105F10004161FDF78BFA08B1012010BD0449044826
:105F20007C31FDF709FA002010BD0000007000521E
:105F30003405002410B58CB004460120ADF82C00C7
:105F40002068FFF7A1FE002853D0A06B032841D0A2
:105F50002068FFF765FC002849D120680021FFF781
:105F600097FEE06604212068FFF792FE2067082173
:105F70002068FFF78DFE60670C212068FFF788FE20
:105F8000A067A06B032825D020680BA9FFF7A7FC0A
:105F900000282CD1A06B03281CD0BDF82C00606415
:105FA00001042068FFF752FC002820D1206800215E
:105FB000FFF76EFEE06504212068FFF769FE2066AA
:105FC00008212068FFF764FE60660C212068FFF757
:105FD0005FFEA06604212068FFF75AFE000D6946A7
:105FE00020642046FDF7CAF830B14FF080500CB065
:105FF00010BD4FF08060FAE7B4F8440000230204BB
:106000002068FFF7F3FBF2E72DE9F84F002604467E
:106010003746354600960068FFF752FB00281FD12F
:106020002068FFF777FB4FF0010808B1E66301E055
:10603000C4F83C8000212068FFF7E2FA4FF0805955
:106040004FF6FF7658B917E020680021FFF7D8FA1D
:10605000002805D120685146FFF7EBFA10B14846F9
:10606000BDE8F88F20680021FFF712FEC50F074634
:106070000098401C009002E0DFF820A00098B04299
:1060800001D2002DE0D0B04202D34FF08070E7E79C
:10609000780001D5C4F838800020E1E7000010C185
:1060A000F8B50D4C164607460D46FAF700F90B48B1
:1060B00033462A4639460094FDF76EFA054603E05A
:1060C000641E01D2012503E0FFF78AFE0028F7D104
:1060D000FAF7EFF82846F8BD00E1F505340500248D
:1060E0002DE9F04186B00D460446FAF7FFFD002188
:1060F00007462068FFF7CCFD800104D54FF400600F
:1061000006B0BDE8F08120684021FFF7A8FAD8B9B1
:10611000B4F8440001042068FFF772FAA0B94FF008
:10612000FF300090402001906020029002200390F8
:10613000002004900120059020686946FFF773FC59
:106140002068FFF7E5FB98B1616B6163D8E7406BAE
:10615000000407D500262068FFF7B8FD761C082E3E
:1061600001C5F8D3FAF7C2FDC01B401C02D126E0DE
:106170004FF000482068416B11F4957FE7D0416BE8
:10618000090701D50820BBE7416B890701D502202B
:10619000B6E7406B800609D52020B1E7FFF796FDF2
:1061A00001C5FAF7A3FDC01B401C08D02068416B55
:1061B0008904F3D42168034888630020A0E740469F
:1061C0009EE700003A0F0018F8B50D4C164607463A
:1061D0000D46FAF76CF80B4833462A4639460094C8
:1061E000FDF7ACFA054603E0641E01D2012503E089
:1061F000FFF7F6FD0028F7D1FAF75BF82846F8BD5F
:1062000000E1F5053405002410B5154C07211348AD
:106210004FF0007204F1080320604FF480006060CA
:10622000002083E80700521062619200A261CA0751
:10623000606362650A07C4E907206062C4E90A0175
:106240002046FDF757FB2068016841F0010101601D
:10625000BDE81040FF2000F005B800000038004005
:10626000405B042401B582B04FF47A7001230090A2
:1062700001AA034802A9FDF75FFC9DF804000EBDCA
:10628000405B04240A4A11680B6823F001030B6089
:1062900011688B6823F0E0438B6011688B680343BF
:1062A0008B601068016841F00101016070470000D7
:1062B000405B042410B502685169936943F00803F8
:1062C00093610268936943F0100393610268136855
:1062D00023F0010313600268136940F26B34A34397
:1062E00013610268936823F44043936090F881201F
:1062F000042A0CD08A060AD5D0F8842042F0800205
:10630000C0F884200268936943F02003936190F8F9
:106310008120032A1DD04A060AD5D0F8842042F0F5
:106320000402C0F884200268936943F0400393613B
:10633000826AB2F5800F0CD10A060AD5D0F8842003
:1063400042F00202C0F884200268936943F080039F
:1063500093618A050AD5D0F8842042F00102C0F882
:1063600084200268936943F400739361C9050AD5D8
:10637000D0F8841041F00801C0F8841001688A69DF
:1063800042F480728A610021A0F86210A0F86A10BD
:1063900010BD2DE9F0411E4617460D468046069C6D
:1063A0000AE0601C08D024B1FAF7A0FC801BA042D0
:1063B00002D90320BDE8F081D8F80000406935EA31
:1063C000000004D00020B842EBD00020F2E701200A
:1063D000F9E7000030B589B014460D4610B1012828
:1063E0000FD105E04FF4007010804001086008E014
:1063F00005486946FCF7A0FF0698401E28600798EC
:10640000208009B0002030BD3405002400B589B0DB
:1064100004486946FCF790FF0698002800D0012048
:1064200009B000BD3405002410B5002410B10128C6
:1064300006D102E001F084FF02E0FFF75DFD0446B3
:1064400060B210BD034900200A7842F010020A70C1
:106450007047000038010024002070472DE9F0410A
:10646000114D0E4600241746297841F0020129708B
:1064700010B1012814D108E04FF6FF7000EA432262
:106480003046790201F0A2FF0AE01A46394630464A
:10649000FFF706FE44B21CB1287840F008002870CF
:1064A0002046BDE8F0810000380100242DE9F041CC
:1064B000114D0E4600241746297841F0010129703C
:1064C00010B1012814D108E04FF6FF7000EA432212
:1064D0003046790201F0E8FF0AE01A4639463046B4
:1064E000FFF772FE44B21CB1287840F00400287017
:1064F0002046BDE8F081000038010024704700000C
:106500002DE9F04F93B01F4615468A460446814652
:10651000580700D0012000EBD7000C2F10FB07F02C
:10652000C0B2129003D0102F01D0182F2FD10246E5
:1065300069462846FAF74FFA002024E01DF8086063
:106540000025DFF850B0300601D51C9A03E01D98F5
:1065500028B9BBF8002051462046FDF707FF70061A
:10656000641CA4B2060EA4EB0900B84204D10AF1DF
:1065700001004C461FFA80FA6D1CEDB2082DE2D3E3
:1065800008F10100C0B2129980468842D6D313B0F8
:10659000BDE8F08FA60100242DE9FF4F83B09B4694
:1065A0000E46044680468A46DDE910750020814685
:1065B0001FE0B9F1000F22D005994FF0000908EB58
:1065C0000100401BA04202DA7019444686B20AEB71
:1065D0000B00401BB0420FDBDDE912012B463A46AF
:1065E000CDE9000131462046FFF78AFF601984B2E9
:1065F000BF1C3A78002ADCD107B0BDE8F08F802AB2
:1066000001D90120D3E7059908EB0100A0EB550063
:10661000A04202DA7019444686B20AEB0B00401B16
:10662000B042E9DB0D2A0DD0DDE912012B46CDE9A0
:10663000000131462046FEF721F804EB550084B2F4
:106640007F1CD6E77019444686B27F1CF5E7000030
:1066500070B5294C9CB0256825F004052560264CB2
:1066600000260C34256845F440452560256805F46E
:1066700040451B952568AD04FCD5212400944FF4BA
:106680008034019401240396CDE90646022409943E
:10669000CDE90A410CAD12960824CDE9104685E8F3
:1066A0000D006846FCF794FA00B1FEE73F20139016
:1066B0000320CDE9140640200101CDE91640CDE9C3
:1066C000180150201A90022113A8FCF7D3F800B14A
:1066D000FEE70A48016841F0800101600748F43094
:1066E000016841F002010160006800F002001B90A7
:1066F000FAF7F6F91CB070BD0C4802580044025875
:10670000FAF7FABA1C48016841F4700101601B49AC
:10671000086840F001000860184A0020103210603C
:106720000A68174B1A400A60144A18321060121D8A
:106730001060121D1060114A28321060121D106086
:10674000121D1060121D1060121D1060121D1060CD
:10675000121D1060121D10600A6822F480220A6067
:1067600006496031086001200649C1F80801C006E9
:10677000014980390860704788ED00E00044025804
:106780007FEDF6EA0080005190F83410C90706D07A
:1067900001684A68836B22F400321A434A6090F819
:1067A0003410890706D501684A68C36B22F4803229
:1067B0001A434A6090F83410490706D501684A68C0
:1067C000036C22F480221A434A6090F834100907BF
:1067D00006D501684A68436C22F400421A434A60B5
:1067E00090F83410C90606D501688A68836C22F4D3
:1067F00080521A438A6090F83410890606D50168E1
:106800008A68C36C22F400521A438A6090F83410EC
:10681000490611D501684A68036D22F480121A43B3
:106820004A60016DB1F5801F06D101684A68436D69
:1068300022F4C0021A434A6090F83410090606D5C3
:1068400001684A68806D22F4002202434A60704762
:10685000F8B500250446C567FAF748FA07462068E8
:1068600000686FF07E46000708D500223B464FF4D3
:1068700000112046009600F0FBFA60B9206800681D
:1068800040070AD500223B464FF48001204600967F
:1068900000F0EEFA08B10320F8BD202084F879005A
:1068A00084F87A00002084F87850F8BD10B5806B29
:1068B0000021A0F86A10A0F86210FDF7EAFA10BDF6
:1068C00001680A6822F490720A6001688A6822F0FE
:1068D00001028A60202180F87A10704710B5B0F864
:1068E0006C2090F87A300168222B05D0088B40F09C
:1068F00008000883022010BD898C8368B3F5805F8F
:1069000001D103696BB11140426E531C4366117093
:10691000B0F86A10491E0904090CA0F86A1007D0E3
:1069200015E0436E11401980416E891C4166EFE706
:1069300001680A6822F490720A6001688A6822F08D
:1069400001028A60202180F87A10FDF733FC0020D4
:1069500010BD00002DE9F04F044600688025FD4B76
:106960000021D4F810C087B0A6680F46D4F81C8068
:1069700046EA0C06D4F814C0A26A4CEA080C46EAAF
:106980000C0632430668DFF8D0C306EA0C0616434D
:10699000066020684268E66822F440523243426052
:1069A0002268A0699A4201D0266A3043A66AB6F1ED
:1069B000005F04D1D4E90B6C46EA0C0630439668BC
:1069C000DFF898C306EA0C06064396602068C26AA0
:1069D000666A22F00F023243C262E14E2068E14A49
:1069E000B04210D1126802F03802182A74D005DCC7
:1069F000CAB3082A7AD0102A47D179E0202A7BD05E
:106A0000282A7CD17AE0D84EB04209D1126802F02F
:106A10000702062A73D2DFE802F053696B6D6F71CB
:106A2000D24EB04209D1126802F00702062A66D29D
:106A3000DFE802F0465C5E606264CD4EB04209D190
:106A4000126802F00702062A59D2DFE802F0394F35
:106A500051535557C74EB0420BD1126802F007028E
:106A6000062A4CD200E00EE0DFE802F02A40424461
:106A70004648C14EB04209D1126802F03802182AC5
:106A800038D0BBDCB4E74FF0010538E0BB4EB04274
:106A900009D1126802F00702062A30D2DFE802F0BC
:106AA0001026282A2C2EB64EB0420BD1126802F0C6
:106AB0000702062A23D2DFE802F003191B1D1F215B
:106AC00000251CE098421AD1A64A121D126802F055
:106AD0000702062A13D202E00CE007E00CE0DFE830
:106AE00002F0030507090B0D022508E0042506E066
:106AF000402504E0082502E0102500E02025DFF80D
:106B000064B2A04E9842DFF880A2ABF1540B73D16F
:106B1000102D31D006DC022D09D0042D0AD0082D0D
:106B20002FD111E0202D29D0402D2AD107E0FBF7ED
:106B300037F913E06846FBF749F901980EE003A81E
:106B4000FBF7C2F9049809E0DBF800105846890603
:106B500010D50068C0F3C1012AFA01F0002811D055
:106B60006168894601EB410181420AD8B0EB093FD7
:106B700007D808E05046F3E78448F1E74FF40040B7
:106B8000EEE7012733E1102D4FF000084ED006DC70
:106B9000022D0FD0042D15D0082D04D12DE0202D6D
:106BA0004AD0402D13D00127794AA0F54071914277
:106BB00070D9E6E7FBF7F4F8626A0023414636F83D
:106BC00012200DE06846FBF701F9019803E003A8E5
:106BD000FBF77AF904980023616A36F81120194608
:106BE000F9F77EFB62680902030241EA106150086E
:106BF000181841EB080115E032E0DBF800105846A8
:106C0000890609D500680023C0F3C1012AFA01F002
:106C1000616A36F8112015E0606A002336F810200A
:106C200050460FE00023F9F75BFBBDE7606A0023E5
:106C300036F81020554805E0606A002336F8102029
:106C40004FF400400021F9F74BFB0902020241EA30
:106C500010614FEA590010184A4641EB0801E1E77C
:106C6000E3694FF4004293424DD1082D23D005DC57
:106C70008DB1012D12D0042D06D112E0102D35D08A
:106C8000202D3AD0402D11D0012721F00F00C1F363
:106C9000420108435AE0FBF7F3FE16E0FBF706FF5C
:106CA00013E06846FBF792F801980EE003A8FBF7A3
:106CB0000BF9049809E0DBF800105846890608D55E
:106CC0000068C0F3C1012AFA01F0616A36F81110B8
:106CD00010E0606A36F81010BAFBF1F0410060680D
:106CE00001EB5001B1FBF0F081B2CEE7606A36F8FB
:106CF00010102648B0FBF1F0F0E7606A36F810009B
:106D0000B2FBF0F0EAE7082D4AD00ADC0DB3012D02
:106D100043D0042D7FF44DAF6846FBF757F8019838
:106D200009E0102D52D0202D55D0402DF2D103A8CE
:106D3000FBF7CAF80498616A36F81110B0FBF1F15C
:106D4000606801EB5001B1FBF0F080B22168C860CF
:106D50004DE01FE0000C0058F369FFCFFFF4FF1176
:106D600000100140544402580044004000480040D4
:106D7000004C0040005000400014014000780040EA
:106D8000007C0040448D00080090D00300093D00C5
:106D9000FFFC0F00FBF774FECDE7FBF787FECAE7A9
:106DA000DBF80020594692060AD50968C1F3C102F2
:106DB0002AFA02F1626A36F81220B1FBF2F20FE011
:106DC000616A36F81120BAFBF2F209E0616A36F81E
:106DD00011200949F1E7616A36F81110B2FBF1F2AE
:106DE000616802EB5102B2FBF1F189B2C16007B0F8
:106DF0003846BDE8F08F000000093D0090F879109A
:106E0000212901D002207047B0F8621021B18168B9
:106E1000B1F5805F13D014E001680A68920004D5D0
:106E20008A6822F400028A6003E00A6822F0800285
:106E30000A600068016841F0400101600CE00169EE
:106E400061B1C16D4A1CC265026809781185B0F84C
:106E50006210491EA0F8621000207047C16D0268E0
:106E60000988C1F308011185C16D891CC165EEE770
:106E70002DE9F0411E46174688460446069D1CE053
:106E8000681C1AD025B1F9F731FF801BA84214D92C
:106E90002068016821F4D07101602068816821F0C8
:106EA00001018160202084F8790084F87A000020B4
:106EB00084F878000320BDE8F0812068C16938EAD1
:106EC000010004D00020B842DAD00020F3E701200E
:106ED000F9E7000070B50D4D00240D48FCF7E0FF08
:106EE00002E0641CAC4204D80948FCF7D3FF202818
:106EF000F7D1002402E0641CAC4206D80549012207
:106F00000348FDF703F90028F5D170BDFFFF01002C
:106F1000B40400240C00002410B5D0F814225268E8
:106F20009047002010BD13460A46002110B500F01E
:106F3000F5F9002010BD13460A46002110B500F0F7
:106F400079FA002010BD10B58021044600F05BFAEC
:106F50002046BDE81040002100F055BA052100236D
:106F600010B51A46C0F8F411194600F0D7F9002000
:106F700010BD10B582610223C0F8F4311346C2611E
:106F80000A46002100F056FA002010BD042100231B
:106F900010B51A46C0F8F411194600F04BFA00205B
:106FA00010BDF8B5044648880D46010A08294BD2A1
:106FB000DFE801F04A0409174A4A4048D4F81012A1
:106FC000207C0A6832E0207C02260028D4F81402D3
:106FD00005D0C16A684688470146467041E0816A2B
:106FE000F8E7C0B206282FD2DFE800F003080D1240
:106FF000171CD4F81012207C4A6817E0D4F810123D
:10700000207C8A6812E0D4F81012207CCA680DE057
:10701000D4F81012207C0A6908E0D4F81012207C01
:107020004A6903E0D4F81012207C8A6969469047C7
:10703000014616E0207C38B9D4F81402416B68464A
:107040008847F5E7207C20B129462046FFF77BFFE3
:10705000F8BDD4F81402016B684688470146072042
:107060004870BDF800000028F2D0EA88002AEFD06E
:10707000824200D902462046ADF80020FFF779FF92
:10708000F8BD002370B500281DD00025044602E09D
:107090006D1C641CEDB22678002EF9D1022404EB9D
:1070A00045041480CC545B1C03220024CA545B1C8E
:1070B00006E0CA545B1CDAB28C54521C401CD3B29A
:1070C0000278002AF5D170BD10B580B1D0F8143225
:1070D00013B10023C0F8143209B1C0F81012012115
:1070E00080F8FC11027000F0CFF8002010BD05A060
:1070F00001F0A0FA05A001F09DFA0AA001F09AFAA9
:10710000022010BD4552524F523A2000496E76611E
:107110006C6964204465766963652068616E646C9F
:10712000650000000D0A000010B5D0F82002F9F744
:107130004BFF002010BD10B5D0F82002F9F722FF58
:10714000002010BD2DE9F0411746044641B1D4F8A6
:10715000140242698AB394F8FC01032842D043E048
:10716000D4F8F411002504F11400022933D1D0E938
:1071700002639E4207D9F31A39469AB283602046C9
:10718000FFF7D9FE12E04068B0FBF3F103FB1101F9
:10719000A1B9984212D3D4F8F81188420ED2002235
:1071A00020461146FFF7C7FEC4F8F85100231A46DF
:1071B0001946204600F0B2F80DE012E0D4F81402AF
:1071C000C16829B194F8FC01032801D12046884701
:1071D0002046FFF7C3FE94F80002012804D184F88A
:1071E000005201E0204690470020BDE8F08170B5D4
:1071F0001546044641B1D4F8140282693AB394F8B2
:10720000FC01032824D025E0D4F8F41104F58270A1
:1072100003291FD1D0E902318B420BD95B1A83605D
:107220000846834200D3034629469AB22046FFF718
:107230007AFE0FE0D4F81402016929B194F8FC0138
:10724000032801D1204688472046FFF79FFE01E032
:1072500020469047002070BD0020704710B50121E6
:1072600080F8FC11D0F81422017952689047002070
:1072700010BD10B5D0F82002F9F7CEFE002010BDE9
:10728000D0F82002F9F7E2BE14494023124A10B5A3
:107290000A6008224A6000220A634B6102230A62E4
:1072A000C1E90632CA62CB608A62C1F8FC03C0F849
:1072B00020120846FAF738FA08488021F9F7FFFD4E
:1072C000064840220021F9F7FEFD044880220121F2
:1072D000F9F7F9FD002010BD0000084040560424D5
:1072E0000A06D0F8200201F07F01C1EBC10100EBDA
:1072F000810002D590F83A00704790F8FA01704783
:10730000002070470020704710B51C46D0F82002BE
:1073100013462246F9F7A4FE002010BD10B5D0F8A0
:107320002002F9F7C7FE002010BD70B50022044608
:1073300040231146FFF7E8FF4025204600222B4658
:107340008021C4F81051FFF7DFFF2562012084F887
:10735000FC01D4F8180228B1D4F81402217942684B
:1073600020469047002070BD90F8FD1180F8FC1178
:107370000020704710B590F8FC11032904D1D0F813
:107380001412C96901B18847002010BD01740020A2
:1073900070470000044B012210B51A70D0F820028B
:1073A000FAF7D0FA002010BDEB00002470B50446B7
:1073B00000F50270054600F092F90120C4F8F401CE
:1073C000B4F80E02C4F8F80194F8082212F01F0075
:1073D0000AD001280DD0022810D002F080012046EA
:1073E00000F011F8002070BD2946204600F0FBF99E
:1073F000F8E72946204600F0DDFAF3E72946204663
:1074000000F06AFAEEE710B5D0F82002F9F776FE40
:10741000002010BD10B5D0F82002FAF7ACFA002019
:1074200010BD90F8FC1180F8FD11042180F8FC11CA
:107430000020704710B5D0F82002F9F78FFE002029
:1074400010BD000004A00A46024910B5FFF719FE5E
:10745000004810BD405A04244D534320436F6E66CC
:107460006967000010B5FDF7D2FA002010BD10B515
:10747000FDF7EBFA002010BD10B501210446FFF71F
:107480005AFE81212046FFF756FE2046FDF7FAFA04
:10749000D4F8181229B1002001F00EFC0020C4F825
:1074A0001802002010BD000012200880004870471C
:1074B0000C0100240A21018000487047E0000024EC
:1074C0002021018000487047A00000242021018075
:1074D0000048704780000024202101800048704748
:1074E000C000002470B50546007C0024C0B14023D4
:1074F000284602220121FFF707FF402328460222E7
:107500008121FFF701FF002048F26C0101F0E0FB50
:10751000C5F8180270B12846FDF7B9FA204670BDCB
:107520004FF400762846022233460121FFF7ECFE95
:107530003346E3E70124F1E704A00A46024910B507
:10754000FFF79FFD004810BD405A04244D534320CF
:10755000496E7465726661636500000004200880EE
:10756000004870470801002404A00A46024910B5EB
:10757000FFF787FD004810BD405A042453544D695D
:1075800063726F656C656374726F6E69637300001C
:107590000A46054910B520B104A0FFF772FD024864
:1075A00010BD08A0F9E70000405A04244D61737330
:1075B0002053746F7261676520696E204653204DB9
:1075C0006F6465004D6173732053746F72616765FA
:1075D00020696E204853204D6F64650009B1C0F8E2
:1075E0001C1200207047000010B51A2008800948BE
:1075F000D0E900148068081809D007490822FCF770
:1076000007FE0549042220461031FCF701FE02481E
:10761000801E10BD0010005C2001002470B5D0F861
:107620001852064608780C4610F0600126D0202932
:1076300053D16178FE2902D0FF2919D10EE061886B
:10764000B1B9E188012913D1000611D5D6F81C0281
:107650008069804701222946286019E0618839B98C
:10766000E18829B9000603D43046FDF734FA34E046
:1076700021463046FFF767FC022070BD6078012884
:107680000DD00A2802D00B2827D105E00122291DA0
:107690003046FFF76EFC20E0A07868601DE021799D
:1076A0003046FFF7E6FD21793046FFF744FD2079AB
:1076B0004FF400730006307C04D500B14023022251
:1076C000812103E000B14023022201213046FFF76F
:1076D0001BFE21793046FDF785F9002070BD0A7840
:1076E00002704A784270CB788A7802EB032242809B
:1076F0004B790A7902EB032282808A79C97902EBFD
:107700000121C180704700000246002010B511B170
:10771000C2F8141210BD05A000F08CFF05A000F007
:1077200089FF0AA000F086FF022010BD4552524F8B
:10773000523A2000496E76616C696420436C617333
:10774000732068616E646C65000000000D0A000023
:1077500010B5D0F8142202241AB11268904700B96B
:107760000024204610BD000070B51B4E0D468978E0
:1077700004460129317028D894F8FC01022802D06F
:10778000032822D105E099B16160032084F8FC014F
:1077900009E091B1606888420AD0C1B22046FFF783
:1077A000BBFB317861602046FFF7D2FF02280CD086
:1077B0002046BDE87040FFF7E9BB022084F8FC01D9
:1077C00020466160FFF7A8FBF2E729462046BDE8A6
:1077D0007040FFF7B8BB0000EA00002410B5FFF7C7
:1077E00019FE002010BD2DE9F0414A78002701263E
:1077F0003B460A2A43D2DFE802F03C584251420895
:1078000005422A27FFF7CDFB63E004468888C8B904
:10781000C888B8B9887800F07F0594F8FC0103287F
:1078200010D02946204684F8FE51FFF7B3FD2046CC
:10783000FFF7ACFB1DB1022084F8FC0149E084F89D
:10784000FC6146E020461AE0FFF78EFF41E0CA885F
:10785000012A14D190F8FC21022A02D0032A0ED169
:1078600004E00122836000F1080114E00122011DFF
:1078700011E090F8FC21022A04D0032A02D0FFF77D
:1078800062FB26E0C660D0F8041209B10321C16092
:10789000022200F10C01FFF76CFB1AE00446488855
:1078A000012816D1C4F804620BE0044690F8FC01EC
:1078B000022801D00328C5D14888012809D1C4F87D
:1078C0000432D4F814028268204690472046FFF71D
:1078D0005DFB3846BDE8F08170B50D460446097978
:1078E00000262878C0F34110012806D06878A0B39C
:1078F00001281FD003283FD107E0D4F814022946FD
:10790000826820469047002070BD94F8FC01022850
:1079100017D003282CD1688828B921B1802902D03A
:107920002046FFF770FDD4F81402294682682046ED
:10793000904713E094F8FC01022802D0032817D1E5
:1079400003E0C9B180291BD116E06888A0B94806B8
:1079500004D02046FFF7E8FBE5E703E02046FFF709
:1079600015FB09E094F8FC01022807D003280BD08E
:1079700029462046FFF7E7FA304670BD4806FBD09F
:107980002046FFF740FDF7E7080601F07F0004EB13
:10799000001501D5143501E005F582752046FFF785
:1079A0009FFC00B101202946022228602046FFF7F3
:1079B000E0FAE1E770B5054690F8FC010C460328B3
:1079C0000DD1207901280AD8D5F8140282682846FA
:1079D0009047E08830B92846FFF7D8FA02E02846F9
:1079E000FFF7B1FA002070BD30B54C781D4B012275
:1079F0000D78AA40012CD0F81C4818D044EA024265
:107A0000C0F81C280A7800EB4210D0F8002B1204B2
:107A10000BD4D0F8002B0C89C4F30A042243C97894
:107A200043EA81410A43C0F8002B002030BD92B2E6
:107A30001443C0F81C480A7800EB4210D0F8004903
:107A40002404F2D4D0F800490D89C5F30A052C436B
:107A5000C978890441EA82510C431C43C0F80049AB
:107A6000E3E7000000800010D0F800196FF30A016E
:107A7000C0F80019D0F80818C1F34101022905D156
:107A8000D0F8001941F00301C0F80019D0F804182B
:107A900041F48071C0F804180020704770B50446A6
:107AA000049D0D99069801280CD0E06840F0400034
:107AB000E060204600F028F84FF48030A063012DEC
:107AC00016D01DE0A06B20F48030A063E0680D4A62
:107AD0001040E060E06820F44010E060012903D12C
:107AE000E06840F48010E060204600F00DF8E6E722
:107AF000A06840F00C00A060A06840F02000A060EA
:107B0000002070BDBFFFBDFF00210B4A491C914200
:107B10000AD80369002BF9DA0021036943F0010355
:107B20000361491C914201D9032070470369DB07B7
:107B3000F7D1002070470000400D030030B54D78AC
:107B400001230C7803FA04F2012DD0F83C4816D03A
:107B500024EA0242C0F83C28D0F81C280C78A34044
:107B600022EA0342C0F81C28097800EB4110D0F843
:107B7000001B21F40041C0F8001B002030BD92B270
:107B80009443C0F83C48D0F81C280C78A3409BB222
:107B90009A43C0F81C28097800EB4110D0F800196E
:107BA00021F40041C0F80019E7E710B5D0F8041837
:107BB00021F00201C0F804180320F8F77FFF00202D
:107BC00010BD10B5D0F8041841F00201C0F8041837
:107BD0000320F8F773FF002010BD00002DE9F047E7
:107BE0000D460446DDE90A1A0027DDF83C80089EB0
:107BF000806B40F40010A063B8F1000F0BD1A06BB4
:107C000020F40010A063206840F04000206020684D
:107C100040F0800020604FF00009C4F8009ED4F8C6
:107C20000008C4F80008012904D0D4F8000840F086
:107C3000030004E0D4F800080BB140F00100C4F8E0
:107C400000081021204600F0BDFA204600F0AAFAF4
:107C50004A46C4F81098C4F814984FF0FF30C4F89E
:107C60001808C4F81C984FF090434FF0FF0C0FE039
:107C700004EB4710D0F80019002902DAC0F80039E7
:107C800001E0C0F80029C0F81029C0F808C97F1C1D
:107C9000BD42EDD800210FE004EB4110D0F8007B8D
:107CA000002F02DAC0F8003B01E0C0F8002BC0F85A
:107CB000102BC0F808CB491C8D42EDD8D4F8100821
:107CC00020F48070C4F81008012E0AD11448C4F8BA
:107CD0003008D4F8300813490843C4F83008D4F801
:107CE0003008A2616FF0804060611EB9A06940F069
:107CF0001000A061A0690C490843A061BAF1000F0F
:107D000003D0A06940F00800A061B8F1010F03D1D1
:107D1000A06906490843A0610020BDE8F087000083
:107D2000000400020300010800383C800400004009
:107D3000816821F0010181600020704730B54D78E5
:107D40004D4C0B7800EB4313012D28D0D3F8105B7A
:107D50006FF31205C3F8105B0B7800EB4313D3F8F5
:107D6000105B2540C3F8105B4B690BB18B684B610E
:107D70000B7800EB4313D3F8104B44F40024C3F802
:107D8000104B0B7800EB4313D3F8104B8D68C5F301
:107D900012052C43C3F8104B012A5BD060E04D69FB
:107DA000002DD3F810593AD06FF31205C3F81059CB
:107DB0000B7800EB4313D3F810592540C3F8105942
:107DC0004C698B689C4200D94B610B7800EB4313E4
:107DD000D3F8104944F40024C3F810490B7800EBA1
:107DE0004313D3F810494D69C5F312052C43C3F86A
:107DF0001049012A27D04A693AB1D0F834280C78C2
:107E00000123A3401A43C0F83428097800EB41103D
:107E1000D0F8001941F00441C0F8001929E02540CC
:107E2000C3F810590B7800EB4313D3F8104944F40E
:107E30000024C3F810490B7800EB4313D3F8104922
:107E40006FF31204D3E70B7800EB43130A69C3F80E
:107E50001429DAE70B7800EB4313CA68C3F8142B34
:107E6000097800EB4110D0F8001B41F00441C0F844
:107E7000001B002030BD0000FFFF07E00023C0F81A
:107E8000103BD0F8103B43F40023C0F8103BD0F86F
:107E9000103B43F01803C0F8103BD0F8103B43F000
:107EA000C043C0F8103B012905D1C0F8142B4FF096
:107EB0008021C0F8001B002070474B780A7800EB47
:107EC0004212012B0BD0D2F8003B23F40013C2F86E
:107ED000003BCA78032A17D0022A15D01DE0D2F839
:107EE000003923F40013C2F80039CA78032A01D0FC
:107EF000022A12D1097800EB4110D0F8001941F0A4
:107F00008051C0F8001908E0097800EB4110D0F862
:107F1000001B41F08051C0F8001B002070474B78D7
:107F20000A7800EB4212012B14D0D2F8003B002B50
:107F300005DBD2F8003B23F08043C2F8003B097810
:107F400000EB4110D0F8001B41F40011C0F8001BF9
:107F500000207047D2F80039002B05DBD2F8003939
:107F600023F08043C2F80039097800EB4110D0F8C3
:107F7000001941F40011C0F80019E9E778B54E780E
:107F80006FF06045834C0B7800EB4313012E2FD02C
:107F9000D3F8106B6FF31206C3F8106B0B7800EB7D
:107FA0004313D3F8106B2640C3F8106B4B69002BBA
:107FB0007DD08C6823445B1EB3FBF4F39BB20C783A
:107FC00000EB4414D4F8106B05EAC3452E43C4F803
:107FD000106B0C7800EB4414D4F8105B8E685E4391
:107FE000C6F312031D43C4F8105B012A73D0B2E03C
:107FF0004E6966B3D3F810696FF31206C3F81069BF
:108000000B7800EB4313D3F810692640C3F81069CE
:108010004C698B681C44641EB4FBF3F305EAC3444B
:108020000B7800EB4313D3F810592C43C3F81049D5
:108030000B7800EB4313D3F810494D69C5F31205D3
:108040002C43C3F81049CB78012B16D027E0D3F886
:1080500010592540C3F810590B7800EB4313D3F89F
:10806000104944F40024C3F810490B7800EB431383
:10807000D3F810496FF312040FE00B7800EB4313B1
:10808000D3F8104924F0C044C3F810490B7800EB32
:108090004313D3F8104944F00054C3F81049012A9F
:1080A00012D0CB78012B17D04B692BB300E037E00F
:1080B000D0F834380D780124AC402343C0F834386C
:1080C000CB78012B08D017E00C7800EB44140B6937
:1080D000C4F81439F4E738E0D0F80838DB050B7839
:1080E00000EB4313D3F8004902D444F0005401E0FC
:1080F00044F08054C3F800490B7800EB4313D3F8E5
:10810000004944F00444C3F80049CB78012B3ED128
:1081100000928A8A93B20A78C96800F0E7F836E0DC
:108120000B7800EB4313D3F8104B8D68C5F31205A1
:108130002C43C3F8104B0B7800EB4313D3F8104BD0
:1081400044F40024C3F8104B4FE70B7800EB4313C3
:10815000CA68C3F8142BCA78012A0FD1D0F80828AE
:10816000D2050A7800EB4212D2F8003B02D443F069
:10817000005301E043F08053C2F8003B097800EB64
:108180004110D0F8001B41F00441C0F8001B002052
:1081900078BD0000FFFF07E0816841F001018160C8
:1081A00000207047002110220261054A491C9142BB
:1081B00001D9032070470369DB06F7D4002070471C
:1081C000400D03000022202343EA8111016105498B
:1081D000521C8A4201D90320704703699B06F7D4D9
:1081E00000207047400D03000021D0F8082812F04D
:1081F000060F15D0D0F80828C2F34102012A0CD08E
:10820000D0F80828C2F34102032A06D0D0F80808A3
:10821000C0F34100022802D002E0032100E0022165
:1082200008467047406900F001007047D0F8181800
:10823000D0F81C08084080B27047D0F81818D0F861
:108240001C080840000C7047D0F81038D0F83428CB
:10825000CA4002F0010243EAC21200EB4110D0F81A
:1082600008091040704700EB4111D1F8081BD0F805
:10827000140808407047416980690840704710B58C
:1082800004460023D21C900804F5805403E02268C1
:1082900041F8042B5B1C8342F9D3084610BD10B58E
:1082A000C26822F0C042C260012901D021B107E0BA
:1082B000C16841F0005102E0C16841F08041C160F5
:1082C0003220F8F7FBFB002010BDD0F8002822F484
:1082D000FE62C0F80028D0F800284FF4FE6303EADD
:1082E00001110A43C0F800280020704730B500246F
:1082F000039D65B9DB1C9B0800EB023000F5805044
:1083000003E051F8042B0260641C9C42F9D3002066
:1083100030BDFEE73EB5040300F014F900F0BCF8F0
:108320004FF4406000224FF400518DE807008310A5
:1083300021462020FCF76EFDBDE83E4000F0ACB8C1
:108340001FB5FCF733FD00F021F800F055F80E4999
:108350004880A0F56F41163914D100F0F3F84FF0C2
:108360004071002000900B140246CDE90101014646
:10837000C020FCF74FFD30208DF80C00012103A830
:10838000FCF764FD1FBD0000200000243EB5022064
:1083900000F056F80446800706D400F0D3F8022017
:1083A00044F0020100F01EF9002000904FF48073A9
:1083B00002460146019002903820FCF72BFD02494D
:1083C000012008703EBD000020000024FEB54FF0E3
:1083D000407405464FF400531646A0138DE819006B
:1083E000831008220B20FCF715FD03B03146284608
:1083F000BDE8F040FCF7FCBC1FB5104801784FF415
:10840000005029B14FF0407102918A130B1404E01F
:108410004FF0807102918A130B14CDE900200022E5
:1084200090201146FCF7F6FC022103A8FCF7E0FCC3
:10843000BDF80C0004B040BA10BD000020000024BC
:108440001FB5002101288DF80C1003D0022803D09D
:10845000032803D0052002E0352000E015200D4A56
:10846000127822B14FF040720091131403E04FF0E4
:10847000807200911314CDE9011200221146FCF71D
:10848000C9FC012103A8FCF7B3FC9DF80C0004B063
:1084900010BD00002000002410B50120FFF7D0FF20
:1084A000C007FAD110BD00002DE9F05FC1F30B0643
:1084B000DFF88C800F0B8A46C6F580548146A242B5
:1084C000154600D81446404639034FF480528B4677
:1084D000FFF77CFF002006E0321818F80210FF2991
:1084E00003D1401C80B2A042F6D3A04221D238462C
:1084F000FFF710FF002006E0831919F80020401C48
:1085000080B208F80320A042F6D34FF480525946B7
:10851000404600F02DF8A5420FD0281BA144A244EC
:1085200085B200267F1C4FF48054A542CBD82C4640
:10853000C9E7224651464846EBE7BDE8F09F0000F8
:10854000D405002409480EB5017800200090019060
:10855000029011B14FF4407301E04FF48073002298
:1085600006201146FCF756FC0EBD0000200000243A
:108570002DE9F04107460E46C8B21546C0F5807495
:10858000A24200D814464FF480782246314638463D
:1085900000F00DF8A54208D0281B27442644444685
:1085A00085B2A542F1D82C46EFE7BDE8F081FEB5D3
:1085B00016460C460546FFF7C5FF4FF040724FF4D4
:1085C000005190138DE807008310214600220220FD
:1085D000FCF720FC31462846FCF738FCBDE8FE409D
:1085E000FFF75ABF03B5012883B004D002280BD08F
:1085F00003280BD001200E490A78002142B14FF028
:1086000040720091131407E03120F4E71120F2E7E3
:108610004FF0807200911314CDE90112002211462F
:10862000FCF7F8FB012104A8FCF710FC05B000BD25
:10863000200000240FB4054B10B503A9044A02988A
:1086400000F03CF810BC5DF814FB000081880008C5
:10865000100000240FB4084B10B504A902AA039817
:1086600000F02CF8044602A9002000F0D1F82046C2
:1086700010BC5DF814FB0000118800080907090E02
:10868000002804DB00F1E02080F80014704700F0BF
:108690000F0000F1E02080F8141D704702E008C8C8
:1086A000121F08C1002AFAD170477047002001E06C
:1086B00001C1121F002AFBD1704700002DE9FF4FB6
:1086C00089B09B460446002506E025280BD05A4673
:1086D0000B999047641C6D1C20780028F5D10DB0D3
:1086E0002846BDE8F08F0027B8460122474900E040
:1086F000074314F8013F203B02FA03F00842F7D188
:1087000020782E2819D114F8010F47F004072A28E1
:108710000ED06FF02F022078A0F1300109290CD87B
:1087200008EB880102EB410100EB0108641CF2E751
:108730000A98641C50F8048B0A9020780028CED048
:10874000642808D0692806D075281ED05A460B998F
:1087500090476D1C58E00A994FF00A0901C90A9127
:10876000002802DA40422D2102E0390504D52B21F0
:108770008DF82010012103E0F90704D02021F7E74C
:108780008A4608AE0DE00021FAE70A994FF00A097F
:1087900001C90A91F7E74946F7F7F7FD303106F8C6
:1087A000011D0028F7D1ADEB060000F12009780784
:1087B00001D44FF00108C84502DDA8EB090000E034
:1087C00000208046002706E008A85A46C05D0B99A5
:1087D00090476D1C7F1C5745F6DB04E030205A465D
:1087E0000B9990476D1CB8F10001A8F10108F5DC68
:1087F00005E016F8010B5A460B9990476D1CB9F12C
:108800000001A9F10109F4DC641C65E709280100F5
:108810000A68531C0B6010707047000010B50446C6
:108820000420FBF715FB0148046010BD080000247C
:1088300070B5002405464FF47A7603E0304600F028
:1088400005F8641CAC42F9D370BD000070B54FF060
:10885000E02500216C69094AAB6912685043AA6996
:108860009A42FCD002D2A3EB020302E0A4EB020680
:108870003344194413468142F1D370BD08000024EB
:108880000349CA695206FCD5C2B20A857047000086
:108890000010014000252C46F7F7EAFD04230222D0
:1088A0000521A020FDF7D4FEF8F72EFA4FF4C8708A
:1088B000FFF7B4FF4FF4E13000F020FAFBF7B4FF0C
:1088C000FBF7C2FCFBF7D2FFFBF7BEFDF7F73AFF61
:1088D0004FF6FF70FBF7E8FCFFF732FD002000F0D9
:1088E00073F9022000F070F94FF4784B0A215A46D0
:1088F000102054A3F7F768FE1F221E21102057A353
:10890000F7F762FE1F22322110205AA3F7F75CFE10
:10891000FFF772FDA0F56F41163902D05BA35A46EE
:1089200001E01F225DA346211020F7F74DFEFDF761
:10893000E3FA10B15EA35A460EE06148D0E9061092
:10894000A1FB00100A0D030D42EA003262485DA14E
:10895000FFF780FE604B1F225A211020F7F734FEEC
:108960005E4900225E48FEF7AFFB5E495C48FEF7B9
:10897000CBFE5D495A48FEF731FE5948FEF72EFFFF
:10898000F9F722F84FF4E160FFF752FF574E4FF02E
:10899000000A574F397889452BD03878C00705D061
:1089A0001F228221102053A3F7F70EFE387880078C
:1089B00005D51F228221102052A3F7F705FE387833
:1089C000400702D553A35A4601E01F2255A3AA210E
:1089D0001020F7F7F9FD3878000702D555A35A465D
:1089E00001E01F224FA3BE211020F7F7EDFD97F8FD
:1089F0000090317888450AD03078012816D051A3EC
:108A00001F2296211020F7F7DFFD96F80080641CE6
:108A1000E4B2C82CBED1504800240221F8F75CF91A
:108A20003878C00604D50025012006E04BA3E7E70F
:108A30006D1CEDB20A2D01D95046307087F800A0A8
:108A4000A8E70000202053544D33324837353020FA
:108A500055534220436172642000000020202020F2
:108A600020C7B6C8EBCABDBFAAB7A2CDF820202048
:108A700000000000206D63756465762E74616F627E
:108A8000616F2E636F6D202000000000573235515A
:108A90003634204572726F72210000005350492015
:108AA000464C4153482053697A653A384D4200009C
:108AB00053442043617264204572726F722100003A
:108AC000B0050024534420436172642053697A65E1
:108AD0003A202575204D4200CC030024EC000024F0
:108AE000A80100244800002484010024EB00002495
:108AF000380100245553422057726974696E672EFD
:108B00002E2E00005553422052656164696E672E17
:108B10002E2E00005553422057726974652045720D
:108B20007220000020202020202020202020202033
:108B30002020000055534220526561642020457278
:108B40007220000055534220446973436F6E6E6576
:108B500063746564200000000000025855534220F1
:108B6000436F6E6E656374656420202020000000F2
:108B7000134A70B5131893F8203093B1114B53F882
:108B800020308B421AD90F4B02EB80020C3B53F87A
:108B900020305069B1FBF3F150F82140002003462A
:108BA00008E011688847012070BD55690E18401C07
:108BB00045F82630A042F8DB002070BD022070BDD1
:108BC00024000024748D000830B504460748084D81
:108BD000002150F82400820005EB8400406900F079
:108BE00087F80120291981F8200030BD5C8D00082C
:108BF000240000242DE9F0411E4E002405460F46B6
:108C0000701990F8200010B93168284688474FF055
:108C1000FF326FB3184B53F82510B7FBF1FCB7FBCD
:108C2000F1F001FB1C7101B1401C13490C3951F8E2
:108C30002510491E1CD406EB8506776957F821C01C
:108C4000BCF1000F04D0002484420FD1002206E0C2
:108C5000641CF9E774698F18521C44F8270082429B
:108C6000F8D353F825004843BDE8F081491EE5D507
:108C70001046F9E724000024688D00080C4B002200
:108C800010B50C4C114653F8203004EB800005E081
:108C9000446954F8214004B1521C491C8B42F7D856
:108CA0004FF47A704243B2FBF3F080B210BD000083
:108CB0005C8D000824000024002906D0034A02EB42
:108CC00080029268891AFFF753BF7047240000247E
:108CD00010B50446FFF78EFF411C05D0034901EB98
:108CE00084018968084410BD002010BD24000024C0
:108CF00001E000F8011B521EFBD270470B490A4AE3
:108D000010B5C1E9002000208860C8600861886152
:108D10000C2048610846FBF783F9BDE81040044980
:108D200001220248FBF7F2B900100140B40400240C
:108D30000C000024000000000102030401020304EF
:108D400006070809010002000400060008000A00E6
:108D50000C00100020004000800000010010000006
:108D600010000000C00300004000000040000000B0
:108D700040000000000004000004000000F00000BB
:108D800000000003008083000000000000000000DD
:108D900006000000000000000000000000000000CD
:108DA000000000000000003F400000000000000044
:108DB000003000400030004000000009000BC03DC2
:108DC000000BC03D00090018C024407FE022403164
:108DD000800000180024C01B000D80324001800379
:108DE000801C4027401C80074000401000600000AD
:108DF000000000000000000000000000001F8020B4
:108E00004040200000402020401F8000000000095A
:108E10000006001F80060009000000040004003F57
:108E2000800400040000000010006000000000004A
:108E3000000000040004000400040004000000001E
:108E40000000400000000000000000002001C006FB
:108E5000003800400000001F802040204020401FBC
:108E6000800000000010403FC000400000000018DB
:108E7000C02140224024401840000010802040249F
:108E80004024401B80000002000D0011003FC00183
:108E90004000003C80244024402440238000001FE8
:108EA000802440244034400380000030002000270C
:108EB000C03800200000001B802440244024401BB8
:108EC0008000001C0022C0224022401F80000000C1
:108ED0000000000840000000000000000000000446
:108EE00060000000000000000004000A00110020E3
:108EF0008040400900090009000900090000000045
:108F0000004040208011000A0004001800200023C7
:108F1000402400180000001F802040274029401FE7
:108F2000400000004007C039000F0001C000402091
:108F3000403FC0244024401B8000001F8020402070
:108F40004020403080000020403FC0204020401F93
:108F500080000020403FC024402E4030C000002050
:108F6000403FC024402E00300000000F0010802041
:108F70004022403380020020403FC0040004003FF4
:108F8000C02040204020403FC02040204000000042
:108F900060202020203FC02000200020403FC0242F
:108FA000400B0030C0204020403FC0204000400027
:108FB0004000C03FC03C0003C03C003FC000002058
:108FC000403FC00C4023003FC020001F80204020B5
:108FD0004020401F80000020403FC0244024001853
:108FE0000000001F802140214020E01FA000002041
:108FF000403FC02440260019C0004018C02440242F
:1090000040224031800000300020403FC0204030EE
:1090100000000020003F80004000403F80200020F2
:10902000003E0001C0070038002000380007C03CA7
:109030000007C038000000204039C0060039C020B9
:109040004000002000384007C038402000000030B9
:109050004021C02640384020C00000000000007FB2
:10906000E0402040200000000070000C0003800061
:109070004000000000402040207FE0000000000091
:109080000020004000200000000000001000100040
:109090001000100010001000000000400000000050
:1090A000000000000002800540054003C000402091
:1090B000003FC0044004400380000000000380041F
:1090C0004004400640000000000380044024403F6C
:1090D000C000400000038005400540034000000040
:1090E0000004401FC0244024402000000002E0058E
:1090F0005005500650042020403FC00440040003A7
:10910000C000400000044027C000400000000000F4
:10911000100010041027E00000000020403FC001B4
:1091200040070004C00440204020403FC0004000F1
:1091300040000007C0040007C0040003C000000492
:109140004007C00440040003C00040000003800446
:1091500040044003800000041007F0045004400362
:10916000800000000003800440045007F000100459
:109170004007C00240040004000000000006400553
:1091800040054004C00000000004001F80044000AF
:10919000400000040007800040044007C000400475
:1091A00000070004C0018006000400060001C0079B
:1091B0000001C006000000044006C0010006C00413
:1091C0004000000410071004E001800600040000C5
:1091D00000044005C00640044000000000000004F8
:1091E000007BE040200000000000000000FFF000D5
:1091F000000000000040207BE00400000000004070
:10920000008000400020002000400000000000001E
:10921000000000000000000000000000000000004E
:10922000001FCC000C00000000000000000800300F
:109230000060000800300060000000022003FC1EF7
:1092400020022003FC1E200220000000000E181146
:10925000043FFF10840C78000000000F0010840F02
:109260003800C0077818840078000000780F841058
:10927000C411240E9800E4008400080800680070FF
:1092800000000000000000000000000000000000DE
:109290000007E018182004400200000000400220EF
:1092A00004181807E000000000000002400240011E
:1092B000800FF0018002400240000000800080002A
:1092C000800FF800800080008000000001000D0089
:1092D0000E00000000000000000000000000800000
:1092E00080008000800080008000800000000C0072
:1092F0000C0000000000000000000000000006005C
:109300001800600180060018002000000007F00827
:109310000810041004080807F00000000008040802
:10932000041FFC000400040000000000000E0C10EC
:10933000141024104411840E0C000000000C1810AE
:10934000041104110412880C700000000000E003F6
:1093500020042408241FFC0024000000001F981093
:109360008411041104108810700000000007F00838
:10937000881104110418880070000000001C0010FF
:109380000010FC13001C001000000000000E38113B
:10939000441084108411440E3800000000070008B7
:1093A0008C10441044088807F00000000000000002
:1093B00000030C030C00000000000000000000008F
:1093C0000101060000000000000000000000800114
:1093D00040022004100808100400000220022002AD
:1093E00020022002200220022000000000100408B9
:1093F000080410022001400080000000000E00124E
:1094000000100C106C10800F00000003E00C18130B
:10941000E4142417C4082807D000000004003C030B
:10942000C41C40074000E4001C000410041FFC1191
:1094300004110411040E880070000003E00C1810E1
:10944000041004100410081C10000010041FFC106D
:109450000410041004080807F0000010041FFC1199
:1094600004110417C410040818000010041FFC1194
:1094700004110017C010000800000003E00C1810D1
:1094800004100410441C780040000010041FFC105D
:10949000840080008010841FFC1004000010041061
:1094A000041FFC1004100400000000000300011061
:1094B0000110011FFE10001000000010041FFC111D
:1094C0000403801464181C1004000010041FFC1016
:1094D00004000400040004000C000010041FFC1F22
:1094E0000000FC1F001FFC1004000010041FFC0CF7
:1094F00004030000E010181FFC100007F00808101B
:109500000410041004080807F0000010041FFC10E9
:10951000841080108010800F00000007F0081810E1
:10952000241024101C080A07F2000010041FFC116C
:1095300004110011C011300E0C000400000E1C11AB
:10954000041084108410441C38000018001000100F
:10955000041FFC100410001800000010001FF81079
:10956000040004000410041FF8100010001E001175
:10957000E0001C007013801C0010001FC0103C0095
:10958000E01F0000E0103C1FC000001004180C1683
:109590003401C001C01634180C100410001C001354
:1095A0000400FC13041C00100000000804101C1030
:1095B00064108413041C0410180000000000000054
:1095C000007FFE4002400240020000000030000C1C
:1095D0000003800060001C00030000000040024007
:1095E0000240027FFE00000000000000000000209A
:1095F0000040004000400020000000000100010089
:1096000001000100010001000100010000400040D4
:109610000020000000000000000000000000980191
:109620002401440144014400FC000410001FFC001C
:109630008801040104008800700000000000700030
:10964000880104010401040088000000000070008B
:10965000880104010411081FFC0004000000F80147
:109660004401440144014400C80000000001040119
:10967000040FFC1104110411001800000000D601B1
:10968000290129012901C90106000010041FFC005D
:109690008401000100010400FC0004000001041921
:1096A0000419FC0004000400000000000000030096
:1096B000010101190119FE0000000010041FFC0047
:1096C00024004001B4010C0104000000001004104B
:1096D000041FFC0004000400000000010401FC0160
:1096E00004010001FC0104010000FC010401FC0074
:1096F0008401000100010400FC0004000000F801E6
:109700000401040104010400F80000010101FF004C
:109710008501040104008800700000000000700052
:109720008801040104010501FF0001010401040195
:10973000FC00840104010001800000000000CC0155
:1097400024012401240124019800000000010001EB
:109750000007F80104010400000000010001F80006
:109760000400040004010801FC0004010001800160
:1097700070000C001001600180010001F0010C007C
:109780003001C00030010C01F001000000010401B3
:109790008C00740170018C01040000010101810141
:1097A00071000E00180160018001000000018401B9
:1097B0000C013401440184010C0000000000000091
:1097C00000000001003EFC400240020000000000DA
:1097D000000000FFFF000000000000000040024009
:1097E000023EFC010000000000000000006000805C
:1097F0000080004000400020002000000000000029
:109800000000000000000000000000000000000058
:109810000000000000000000000000000000000048
:1098200000000000000000000000000000000F80A9
:10983000380FFE380F8038000000000000000000E4
:109840000000000000000000000100000600000C05
:1098500000003800003100000600000C0000380055
:10986000003000000000000000000061800067F888
:1098700007F98000618000618000618000618000E4
:1098800067F807F980006180000000000000000018
:109890000001C0E003E0F00630080418081FFFFED6
:1098A000040E080787F00381E000000000000001BB
:1098B000F000060C00040408060C7001F9C0000E4C
:1098C00000003BE000EC18070808040C180003E057
:1098D0000000000001E00007F003F818041C080471
:1098E000170807E1D003C0E00023B0003C080020C7
:1098F000080000100000000000000100003100001E
:109900003200001C00000000000000000000000009
:109910000000000000000000000000000000000047
:1099200000000000000000000000007F0001FFC0F8
:109930000780F00C00181000042000020000000056
:1099400000002000021000040C00180780F001FF46
:10995000C0007F00000000000000000000000000C8
:1099600000000000000000420000660000660000E9
:109970003C0000180003FFC0001800003C00006617
:10998000000066000042000000000008000008001F
:1099900000080000080000080001FFC000080000E7
:1099A0000800000800000800000800000000000097
:1099B0000100003100003200001C00000000000027
:1099C0000000000000000000000000000000000097
:1099D000000000080000080000080000080000085F
:1099E000000008000008000008000008000008004F
:1099F00000000000000000000000003800003800F7
:109A0000003800000000000000000000000000001E
:109A10000000000000000000000000000600001C24
:109A2000000070000180000E0000380000C0000738
:109A300000001C0000300000000000000000007F5B
:109A40008001FFE00380700600180400080400088D
:109A500006001803807001FFE0007F800000000016
:109A6000000000000001000801000801000803FFD9
:109A7000F807FFF8000008000008000008000000D8
:109A800000000000000001C03802C0580400980423
:109A90000118040218040418061C1803F81801E041
:109AA000F800000000000000000001C0E003C0F06A
:109AB00004000804080804080806180803F418013C
:109AC000E7F00001E00000000000000000000003DB
:109AD00000000D0000110000610000810803010872
:109AE00007FFF80FFFF80001080001080000000060
:109AF00000000000E007FCD0060808061008061069
:109B000008061008061838060FF00607C000000007
:109B1000000000000000003F8001FFE003843002ED
:109B20000818041008041008041008071810030F80
:109B3000F00007C000000000000000000003C000AB
:109B40000700000600000600F80607F806180006E1
:109B5000E00007000006000000000000000001E136
:109B6000E003F7F0063410041808041808040C0881
:109B7000040C0806161803F3F001C1E00000000011
:109B8000000000F80003FC30030638040208040259
:109B9000080402080404100308F001FFC0007F005D
:109BA00000000000000000000000000000000000B5
:109BB00000000070380070380070380000000000AD
:109BC0000000000000000000000000000000000095
:109BD00000000000000000301A00301C00000000EF
:109BE0000000000000000000000000000000000075
:109BF00000000800001400002200004100008080E6
:109C000001004002002004001008000800000000CD
:109C1000000000210000210000210000210000219F
:109C2000000021000021000021000021000021008F
:109C300000000000000000000008000804001002FE
:109C4000002001004000808000410000220000143C
:109C50000000080000000000000003C00004C00075
:109C6000040000080038080F380808380810000CF5
:109C7000300007E00003C000000000000000003FCB
:109C80008000FFE0038070020F1006708804C08817
:109C9000048308047F8802C09003012000FE400076
:109CA00000080000180001F8003E0801C200070289
:109CB0000007E20000FE00001FC80001F8000038A5
:109CC00000000804000807FFF807FFF8040808046C
:109CD000080804080804080806180803F41801E72F
:109CE000F00001E0000000000000003F8001FFE004
:109CF000038070020018040008040008040008042F
:109D000000100600200780C000000004000807FFC4
:109D1000F807FFF80400080400080400080400180D
:109D200002001003807001FFE0007F80000000044B
:109D3000000807FFF807FFF80408080408080408EB
:109D400008040808043E0804000806001801006022
:109D500000000004000807FFF807FFF804080804E3
:109D60000800040800040800043E00060000060085
:109D700000018000000000000000003F8001FFE0C3
:109D80000380700600180400080402080402080298
:109D900003F00783F000020000020004000807FF40
:109DA000F807FFF804080800080000080000080091
:109DB00000080004080807FFF807FFF8040008007F
:109DC000000000000004000804000804000807FF69
:109DD000F807FFF804000804000804000800000069
:109DE0000000000000000000060000070000010461
:109DF000000104000104000307FFFE07FFFC04004C
:109E00000004000004000004000807FFF807FFF842
:109E1000040C08001800003E0004C7800503C806B3
:109E200000F804003804001800000804000807FFC8
:109E3000F807FFF804000800000800000800000808
:109E40000000080000080000180000600000000486
:109E5000000807FFF807800807FC00007FC0000328
:109E6000F80007C000780007800807FFF807FFF830
:109E700004000804000807FFF807000803C00000FA
:109E8000E000003800001E000007000001C00400D0
:109E9000F007FFF8040000000000007F8001FFE0F1
:109EA0000380700600180400080400080600180368
:109EB000003001FFE0007F8000000004000807FF81
:109EC000F807FFF804040804040004040004040074
:109ED000040400060C0003F80001F000000000007C
:109EE0000000007F8001FFE003807006008804000E
:109EF000880400C806003C03003E01FFE6007F84A2
:109F000000000004000807FFF807FFF80408080431
:109F10000800040C00040F00040BC00610F003F04E
:109F20003801E00800000800000001E0F803F0300C
:109F3000063010041808041808040C08040C080261
:109F400006180207F00781E000000001800006000B
:109F50000004000004000004000807FFF807FFF8F1
:109F60000400080400000400000600000180000452
:109F7000000007FFE007FFF00400180000080000E1
:109F80000800000800000800000804001007FFE0B7
:109F900004000004000006000007E00007FE0004C3
:109FA0001FE00001F80000380001E0043E0007C097
:109FB0000006000004000004000007E00007FFC0E6
:109FC000041FF80007C007F80007FF80043FF800EF
:109FD00007C004F8000700000400000000000400AF
:109FE0000806001807C07805F1C8003E00001F8071
:109FF0000463E80780F80600180400080000000465
:10A00000000006000007800007E008047C08001F2D
:10A01000F80007F800180804E00807000006000030
:10A020000400000000000100080600380400F804E5
:10A0300003E8040F08047C0805F00807C0080700BF
:10A040001804006000000000000000000000000094
:10A050000000000000003FFFFE2000022000022060
:10A0600000022000022000020000000000000000AA
:10A070000008000007000000C000003800000600D3
:10A080000001C000003000000E00000100000000D0
:10A09000000000000020000220000220000220003A
:10A0A000022000023FFFFE00000000000000000050
:10A0B0000000000000000000000000000800001088
:10A0C00000003000002000003000001000000800F8
:10A0D000000000000000000000010000010000017D
:10A0E000000001000001000001000001000001006B
:10A0F000000100000100000100000100000000005C
:10A1000000000000200000200000100000100000EF
:10A11000000000000000000000000000000000003F
:10A1200000000000F00019F8001B180022080026AB
:10A1300008002408002410003FF8001FF800000861
:10A1400000001800000004000007FFF80FFFF000F7
:10A150001818001008002008002008003018001F00
:10A16000F0000FC00000000000000007C0001FF05A
:10A17000001830002008002008002008003C0800DB
:10A180001C1000006000000000000000000000073C
:10A19000C0001FF000381800200800200800200828
:10A1A00004101007FFF80FFFF0000010000000007F
:10A1B00000000000000007C0001FF0001230002265
:10A1C00018002208002208003208001E10000E208D
:10A1D000000000000000002000002008002008010E
:10A1E000FFF803FFF80620080420080420080720D1
:10A1F0000003000000000000000000000E000E6ED2
:10A20000001FF30031B10020B10020B100319100F6
:10A210001F13002E1E00200E00300000000004005E
:10A220000807FFF80FFFF8001008002000002000CA
:10A23000002008003FF8001FF800000800000000A0
:10A240000000000000002008002008002008063F51
:10A25000F8063FF8000008000008000008000000B1
:10A2600000000000000000000000000300000300E8
:10A270002001002001002003063FFE063FFC0000F5
:10A280000000000000000000000004000807FFF8C4
:10A290000FFFF8000188000300002FC00038F8000D
:10A2A0002038002008000008000000000000000026
:10A2B0000004000804000804000807FFF80FFFF876
:10A2C0000000080000080000080000000000000076
:10A2D0002008003FF8003FF8001008002000003F71
:10A2E000F8003FF8001008002000003FF8003FF899
:10A2F000000008000000002008003FF8003FF800C0
:10A300001008001000002000002008003FF8001F87
:10A31000F80000080000000000000007C0000FF077
:10A320000018300030080020080020080030080025
:10A330001830000FF00007C00000000000000020EF
:10A3400001003FFF003FFF0010110020090020081E
:10A35000002008003038001FF0000FC0000000008F
:10A3600000000007C0001FF000381800200800207F
:10A3700008002009001011001FFF003FFF0000012E
:10A38000000000002008002008002008003FF8001E
:10A390003FF80008080010080020080020000030E6
:10A3A00000003000000000000000000000000C78F9
:10A3B000001E18003308002308002108002188002F
:10A3C00021980030F00038600000000000000020FC
:10A3D0000000200000200000FFF003FFF80020082C
:10A3E00000200800200800003000000000000000ED
:10A3F0000000002000003FF0007FF800001800007F
:10A4000008000008002010003FF8007FF000001056
:10A41000000000000000002000003000003C0000B0
:10A420003F800023F0000078000070002380003C93
:10A4300000003000002000002000003C00003FE051
:10A440000023F80000E0002700003E00003FE0008D
:10A4500021F80001E0003E00002000000000002084
:10A4600008002008003838003E680027800003C834
:10A47000002CF800383800201800200800000000E8
:10A480000000002000003003003C01003F83002357
:10A49000EC000070002380003C0000200000200041
:10A4A0000000000000000000000038080020380014
:10A4B00020F80023E8002F88003E0800380800201C
:10A4C0001800007000000000000000000000000004
:10A4D0000000000000000008000014001FF7FC301E
:10A4E0000006200002000000000000000000000044
:10A4F00000000000000000000000000000FFFFFF5F
:10A50000000000000000000000000000000000004B
:10A5100000000000002000023000061FF7FC0014BD
:10A520000000080000000000000000000000000023
:10A530000000000000001800006000004000004023
:10A5400000002000001000000800000400000400CB
:10A55000000C0000100000B5E70200020002007FBE
:10A56000F0421042107FF0421042107FF042000291
:10A5700008020801F800000000D7D37FF000200097
:10A5800040008001000200FFF80200020002000209
:10A5900000020002000E0000000000BCBC102010F1
:10A5A00020102013FEFC201020102015FC188430F1
:10A5B00088D04810501020105051882606CAF50146
:10A5C000000120011001107FFC03800540054009B7
:10A5D000201110210841040102010001000100D2F4
:10A5E000BA0080404027F811400140827842481666
:10A5F000A81AD02350222042204250028800000096
:10A6000000BEA73FE020203FE020203FE00000FD0B
:10A61000F885088508FDF885088508FDF885080097
:10A62000000000B2E200084F8828880AA88AA84AD9
:10A63000A80AA82AA82AA842284508848888881039
:10A640003800000000CAD44050204820400FF800D5
:10A6500040E04027402240224022202A2833A82ED2
:10A6600018000800000000B3CC00001BF0E210222C
:10A670001023F0F800200033F068806080A3F02001
:10A6800080208027F800000000D0F2020001003F87
:10A69000F820002FF02020224021803FF820882041
:10A6A0009040804080838000000000D1D5200010C1
:10A6B000F87E20444028F87E8848A850A864A8481E
:10A6C000A872A884501888610800000000C9AB1067
:10A6D0000010003FE0404080807FF0421042104276
:10A6E000107FF04000400840083FF800000000CC18
:10A6F000EE20802FF8208027F0F41027F024102778
:10A70000F0241027F03410CFF802200410000000CD
:10A7100000B3E404000200FFF80800104020207F8E
:10A72000F0089008800880088010882088C0780091
:10A73000000000CEC4040002000200FFF810401028
:10A74000400880088005000200050008803060C0D5
:10A750001800000000D7D604000200FFF88008802F
:10A76000083FC0008001000200FFF8020002000262
:10A77000000E0000000000CFD43FE0202020203F4A
:10A78000E0202020203FE008804890289028A00862
:10A79000800880FFF800000000CABE00003FE00013
:10A7A0000000000000FFF8020012401220221042B8
:10A7B00008820802000E0000000000CDBC7FF840B7
:10A7C00008440847C84848548843084CC873384070
:10A7D000884C08430840887FF800000000C6AC00A1
:10A7E000802080208020803FF02000200020003F3B
:10A7F000C02040204020404040804000000000B485
:10A80000A520403840484091F07D50555055507D2E
:10A810005055F054407C40545057F88C08000000CC
:10A8200000C3FE2220222027F8FA2027F024102738
:10A83000F03410E7F020802FF821402220EC18009F
:10A84000000000CAE440804140F22044108BE8A0A0
:10A8500000F78824A827A834A8E7A824A8248825D6
:10A86000B800000000C8EB08000400040002000269
:10A87000000500050008800880104010402020409E
:10A8800010800800000000C8AB02000200050008AC
:10A890008010402020DFD8020002001FC00200020A
:10A8A000000200FFF800000000B3CC00001BF0E243
:10A8B00010221023F0F800200033F068806080A39D
:10A8C000F02080208027F800000000BCBC20802001
:10A8D000802080F7F02080208027E03220E22021B5
:10A8E00040208021402220EC1800000000CAF50220
:10A8F00000024002200200FFF807000A800A8012CE
:10A90000402220421082080200020000000000D60F
:10A91000A702000200FFF8020002007FE0102010F2
:10A9200040088005000200050018C0E03800000063
:10A9300000B3D62080208023F0F880208027F828DC
:10A94000203020E7F82020222021202020E0E000F5
:10A95000000000D7A8020002007FF004000400FFFE
:10A96000F8080010003FE0002000401C80030000B9
:10A970008000000000D7A201004080200017F000F6
:10A980008080804080008017F010802080208040F0
:10A99000804FF800000000C5FA204024402440F415
:10A9A000482450276024403440E44024402440257B
:10A9B000482648E43800000000B7A2020022202206
:10A9C0001044007FF8040008000FE01420244042E7
:10A9D00080810006C0383800000000B3C900A00024
:10A9E0009000807FF8408040907C90449044A04448
:10A9F000A0444858A84118820800000000B9A601E8
:10AA0000000100F90023F021102110211021102154
:10AA1000103910C21002100410086000000000D2AB
:10AA2000C60000002000780CE47904516810307EE4
:10AA30006019981A3C2FE448E408380030006000A0
:10AA400000D1A100000120012003FC622034200479
:10AA50002003FC240021B021202220323E18000FC8
:10AA6000E00000D4F10000000010FC1304110C3DC4
:10AA7000F8703E10D015907CF0503E18101BFE026E
:10AA80003000200000CFEE0000000003FE00607CDC
:10AA90004012FC11041106113611241F44794400A0
:10AAA000C0009C01860000C4BF000000000FE03C15
:10AAB00018200820043E04600460047E0460042022
:10AAC0000C20081FF001800000B6CC000008001127
:10AAD000FC103E3EF82D8C2904490409043E8C509C
:10AAE000FC10881EC811FC100E0000B0B40000005D
:10AAF00040006012FE13023A427F4410C41BFE3C29
:10AB0000987190113011A00078004C0000C8B70077
:10AB100000004000F878C41F8C313821EC21264118
:10AB20003A7DE2272225FA3D26012401040000B6E1
:10AB3000A80000010001705FFC700420042FF801E0
:10AB4000001100113821C431003F0063E04038009B
:10AB500000B3A4000000000818086008C00B001E25
:10AB600000181C7FF01000118010E01838098E0FBB
:10AB7000000000B0B400000040006012FE13023A72
:10AB8000427F4410C41BFE3C987190113011A0000C
:10AB900078004C0000B7B50000000007F80600245C
:10ABA0000014F8078C04042408261825F0647C643B
:10ABB000C220801FC00000BBD8000000001FF03082
:10ABC000182008278C2C44284428442CC42784208F
:10ABD00004300C1FF803800000C7B60100210821D3
:10ABE000083FF800202220223EFF42229422103EFD
:10ABF00010221022283E2822440082CABD004800AC
:10AC00004400440040FFFE004000403E4008400831
:10AC100040082008220F12780A20060002BFAA006E
:10AC2000007FFC08200820082008200820FFFE08DC
:10AC3000200820082008201020102020204020B7C5
:10AC4000A201001110110822003FFC0200040007BD
:10AC5000F80A080908111010A0204040A003181C91
:10AC600006CDF800007FFC40044004421452944A90
:10AC700054442444244A544A5452946104400440A5
:10AC8000144008D6D001000100010001003FF82166
:10AC90000821082108210821083FF82108010001A6
:10ACA0000001000100CEC4020001000100FFFE10FF
:10ACB00010101008200820044002800100028004C7
:10ACC0004008203018C006B2E2000427C41444141F
:10ACD00054855445544554155415542554E5542170
:10ACE000042284224424140808CAD40028202410F2
:10ACF00024102007FE0020F02017E0112011101171
:10AD000010151019CA170A02060002000000000000
:10AD10000000000000000000000000000000000033
:10AD200000000000000000000000000000B4F3007C
:10AD300000000000000018000010000010000010CB
:10AD40000000100000100C3FFFFE00100000180073
:10AD500000180000340000340000220000620000EF
:10AD6000410000C1800080C001006006003808007A
:10AD70001C300000000000D4BD00000000000003F3
:10AD800000C00200B00200980260881F888C020F89
:10AD9000F0020C80022C887FDC88030C901B0CD006
:10ADA0001B0C6013EE60131E64130CF413019C1B48
:10ADB000020C27040421D800407FFC4007F8000063
:10ADC00000B4B400000000000003800803000C027F
:10ADD000E00C06300C04198C08088C08008C182034
:10ADE0008C2FF08C48208C08208C08208C08208C1C
:10ADF00008608C09C10C08080C08080C08080C0C29
:10AE00000C0C07FC78000010000000D0C20000000D
:10AE100000000002000801003C0133C03EC20008EF
:10AE20006200044200048200049A0C3FFFFE01020B
:10AE3000300102300112301FE2300102300D423089
:10AE400019363011143021143021083047103002E7
:10AE50002030000000D2BA00000000000000060010
:10AE60001803000C020C04FDF001198001110042CE
:10AE700033083222F812421812651004E490056A71
:10AE8000B0056A200A71200861403860C01860C0AF
:10AE900018616018623018641E087800000000BE57
:10AEA000A700000000000001004001FFC0010040B9
:10AEB00001004001FFC001004001004001FFC0014E
:10AEC00000400000001064081FE7F8104608104614
:10AED000081046081FC7F810460810460810460814
:10AEE0001FC7F8104608000000C6C100000000009F
:10AEF000000800000FFFF80C00180C00180FFFF8F6
:10AF00000C40900C30C00C10800C11100DFFF80894
:10AF1000308008308008308808309C1FFFE0102007
:10AF2000801020802060802040804080800300804E
:10AF3000000000B2E200000000000011000C09FE59
:10AF4000080D860805864801A64841B64833B6482C
:10AF500013B64815B64805B64805B64805B64809BB
:10AF6000A64809A64839A448182048185808184483
:10AF700008188608190238060018000000CAD40014
:10AF800000000000000001A01001D80800880C009B
:10AF90008804008400FFFE00008000008004008020
:10AFA0003C0280047DC00408C0040840040840043A
:10AFB0004860048822050F3407381406E01C04009A
:10AFC0000E0000060000000000000000000000006D
:10AFD0000000000000000000000000000000000071
:10AFE0000000000000000000000000000000000061
:10AFF0000000000000000000000000000000000051
:10B000000000000000000000000000000000000040
:10B010000000000034B0000800000024A801000077
:10B020001804000834B10008A801002430640400AA
:10B03000AC860008113C90D00304B1320192101587
:10B0400016EFC98B14087D8C140840161224344066
:10B050001FC01620401604241A440C12F04220137C
:10B06000E5741B087904131D7682081A65101A6F9F
:10B0700004C11ACD101AC1041AD9041AB50414094E
:10B0800002202008010104C0320904100A02080647
:10B0900050050705810212022C070501070914203B
:10B0A0002240292019070B1C0907201B0A064521ED
:10B0B0002A40D41AA970135D751B0869041A9104FB
:10B0C0001AE9041A45141A39084F04030904120135
:10B0D0002C158304205700081A02010203011A03E9
:10B0E000358002021F681D44657645426F78202036
:10B0F00053504920466C617368204469736B20315A
:10B100002E30202418084D43554445562024AA4487
:10B11000234924211329641C08D5638C19081A5962
:10B12000041A5D041AAD041A0D0413390122240314
:04B1300000FFFF001D
:040000050800029954
:00000001FF
